:10008C0018810AE00E945B6224E00E9437621F9391
:10009C0018810AE00E945B62102F0F91100F0895D7
:1000AC00188124E00E9447620AE00E9451621F936B
:1000BC0018811F700F91100F08952397F89418E66C
:1000CC0097FC78941F9310E0312FE89490F84F919F
:1000DC00A0E0B0E00E94224E1095112311F40C9474
:1000EC007A0010E00C94C200F89418E697FC78940F
:1000FC001F93FE01A3E0B0E04F910E94104E1095AB
:10010C00112311F40C948D0010E00C94C200EB81BF
:10011C00FC81EF93FF93CF93DF93FE013296108116
:10012C001A930E945600DF91CF91FF91EF9111939A
:10013C00EB81FC813196EF93FF93CF93DF93FE011C
:10014C00319610811A930E945600DF91CF91FF9146
:10015C00EF911193EB81FC813296EF93FF93CF9348
:10016C00DF93FE0110811A930E945600DF91CF910C
:10017C00FF91EF9111931FEF08952497F89418E6CF
:10018C0097FC78941F9313E0312FE89490F84F91DB
:10019C00A0E0B0E00E94224E1095112311F40C94B3
:1001AC00DA0010E00C943401F89418E697FC78947B
:1001BC001F93FE01A4E0B0E04F910E94104E1095E9
:1001CC00112311F40C94ED0010E00C943401EC812B
:1001DC00FD81EF93FF93CF93DF93FE0110811A9370
:1001EC000E945600DF91CF91FF91EF911193EC811A
:1001FC00FD813196EF93FF93CF93DF93FE01319600
:10020C0010811A930E945600DF91CF91FF91EF91CC
:10021C001193EC81FD813296EF93FF93CF93DF9393
:10022C00FE01329610811A930E945600DF91CF91F5
:10023C00FF91EF911193EC81FD813396EF93FF9336
:10024C00CF93DF93FE01339610811A930E945600D0
:10025C00DF91CF91FF91EF9111931FEF08952197AB
:10026C001981173131F020F4103010F0442701C0FF
:10027C0041E010E009F41FEF112311F40C946E010E
:10028C00CF93DF9319811A930E944600DF91CF918F
:10029C001883F89418E697FC78941F9312E01F9338
:1002AC00E89490F8FE01A1E0B0E03F914F910E94DC
:1002BC00224E1095112311F40C94690110E00C944A
:1002CC0071010C946C011FEF0C9471010C94710171
:1002DC0010E00C9471010895219719811B3331F0B2
:1002EC0020F4103010F0442701C041E010E009F474
:1002FC001FEF112311F40C94AB01CF93DF931981F1
:10030C001A930E944600DF91CF911883F89418E657
:10031C0097FC78941F9311E01F93E89490F8FE01DA
:10032C00A1E0B0E03F914F910E94224E1095112315
:10033C0011F40C94A60110E00C94AE010C94A901DC
:10034C001FEF0C94AE010C94AE0110E00C94AE01B6
:10035C000895219719811B3331F020F4103010F0DF
:10036C00442701C041E010E009F41FEF112311F400
:10037C000C94E801CF93DF9319811A930E944600E5
:10038C00DF91CF911883F89418E697FC78941F931B
:10039C0010E01F93E89490F8FE01A1E0B0E03F91CB
:1003AC004F910E94224E1095112311F40C94E301ED
:1003BC0010E00C94EB010C94E6011FEF0C94EB0194
:1003CC000C94EB0110E00C94EB010895188117309C
:1003DC0031F020F4113010F0442701C041E010E05E
:1003EC0009F41FEF112311F40C941B02F89418E676
:1003FC0097FC78941F9313E01F93E89490F8FE01F8
:10040C00A1E0B0E03F914F910E94224E1095112334
:10041C0011F40C94160210E00C941E020C941902A8
:10042C001FEF0C941E020C941E0210E00C941E0282
:10043C000895219719811F3131F020F4113010F0FB
:10044C00442701C041E010E009F41FEF112311F41F
:10045C000C945802CF93DF9319811A930E94460093
:10046C00DF91CF911883F89418E697FC78941F933A
:10047C0014E01F93E89490F8FE01A1E0B0E03F91E6
:10048C004F910E94224E1095112311F40C9453029B
:10049C0010E00C945B020C9456021FEF0C945B0260
:1004AC000C945B0210E00C945B0208952197198167
:1004BC001C3031F020F4113010F0442701C041E021
:1004CC0010E009F41FEF112311F40C949502CF9353
:1004DC00DF9319811A930E944600DF91CF91188304
:1004EC00F89418E697FC78941F9315E01F93E89402
:1004FC0090F8FE01A1E0B0E03F914F910E94224E96
:10050C001095112311F40C94900210E00C949802A5
:10051C000C9493021FEF0C9498020C94980210E028
:10052C000C949802089521971981133631F020F418
:10053C00103010F0442701C041E010E009F41FEF27
:10054C00112311F40C94D202CF93DF9319811A93D7
:10055C000E944600DF91CF911883F89418E697FC1F
:10056C0078941F9316E01F93E89490F8FE01A1E095
:10057C00B0E03F914F910E94224E1095112311F43F
:10058C000C94CD0210E00C94D5020C94D0021FEF09
:10059C000C94D5020C94D50210E00C94D50208955D
:1005AC00CF93DF93FE0110811A930E943501DF91E6
:1005BC00CF911095112311F40C94E70210E00C94D8
:1005CC000C03CF93DF93FE01319610811A930E9496
:1005DC007201DF91CF911095112311F40C94F90253
:1005EC0010E00C940C03CF93DF93FE013296108134
:1005FC001A930E94AF01DF91CF911095112311F442
:10060C000C940B0310E00C940C031FEF0895CF9384
:10061C00DF93FE0110811A930E94EC01DF91CF91C0
:10062C001095112311F40C941E0310E00C94550337
:10063C00CF93DF93FE01319610811A930E941F0213
:10064C00DF91CF911095112311F40C94300310E02D
:10065C000C945503CF93DF93FE01329610811A93BD
:10066C000E945C02DF91CF911095112311F40C9430
:10067C00420310E00C945503CF93DF93FE013396A5
:10068C0010811A930E949902DF91CF91109511233A
:10069C0011F40C94540310E00C9455031FEF0895BF
:1006AC00FE0132961081193010E011F008F01FEFA6
:1006BC00112311F40C948303E881F981EF93FF93D8
:1006CC003196FA93EA931EE01A9317EF91221FEBDF
:1006DC009122FE013596108150E040E0E0E20E944C
:1006EC00345C1EE01F9318810F91011B102FFF919A
:1006FC00EF91108323960C94A503E881F981EF9375
:10070C00FF933196FA93EA931EE01A9317EF912216
:10071C001FEB912210E30E94FE61FE0135961081C1
:10072C0050E040E0E0E20E94345C1EE01F93188130
:10073C000F91011B102FFF91EF9110832396E881ED
:10074C00F981EF93FF933196FA93EA931EE01A9393
:10075C0017EF91221FEB9122EB81FC810E942A5C06
:10076C001AE30E94FE611EE01F9318810F91011B7A
:10077C00102FFF91EF9110832396FE013296319644
:10078C001081193010E011F008F01FEF112311F453
:10079C000C94F603E881F981EF93FF933196FA9369
:1007AC00EA931EE01A9317EF91221FEB9122EB8133
:1007BC00FC810E942A5CFE0135963196108150E036
:1007CC0040E0E0E20E94345C1EE01F9318810F9120
:1007DC00011B102FFF91EF91108323960C941D0495
:1007EC00E881F981EF93FF933196FA93EA931EE037
:1007FC001A9317EF91221FEB9122EB81FC810E943F
:10080C002A5C10E30E94FE61FE0135963196108140
:10081C0050E040E0E0E20E94345C1EE01F9318813F
:10082C000F91011B102FFF91EF9110832396E881FC
:10083C00F981EF93FF933196FA93EA931EE01A93A2
:10084C0017EF91221FEB9122EB81FC810E942A5C15
:10085C001AE30E94FE611EE01F9318810F91011B89
:10086C00102FFF91EF9110832396FE013296329652
:10087C001081193010E011F008F01FEF112311F462
:10088C000C946E04E881F981EF93FF933196FA93FF
:10089C00EA931EE01A9317EF91221FEB9122EB8142
:1008AC00FC810E942A5CFE0135963296108150E044
:1008BC0040E0E0E20E94345C1EE01F9318810F912F
:1008CC00011B102FFF91EF91108323960C9495042C
:1008DC00E881F981EF93FF933196FA93EA931EE046
:1008EC001A9317EF91221FEB9122EB81FC810E944E
:1008FC002A5C10E30E94FE61FE013596329610814F
:10090C0050E040E0E0E20E94345C1EE01F9318814E
:10091C000F91011B102FFF91EF91108323960895D7
:10092C00FE0132961081113011F00C94BF04E88155
:10093C00F981EF93FF933196FA93EA931EE01A93A1
:10094C0017EF91221FEB9122E0E3F0E0B1E0BBBF87
:10095C00B791BB2311F00E94225C1EE01F931881FB
:10096C000F91011B102FFF91EF91108323960C9484
:10097C00A305123011F00C94E504E881F981EF9392
:10098C00FF933196FA93EA931EE01A9317EF912294
:10099C001FEB9122E5E3F0E0B1E0BBBFB791BB23C5
:1009AC0011F00E94225C1EE01F9318810F91011B15
:1009BC00102FFF91EF91108323960C94A305133005
:1009CC0011F00C940B05E881F981EF93FF933196AC
:1009DC00FA93EA931EE01A9317EF91221FEB9122E0
:1009EC00EAE3F0E0B1E0BBBFB791BB2311F00E948A
:1009FC00225C1EE01F9318810F91011B102FFF9199
:100A0C00EF91108323960C94A305143011F00C94E1
:100A1C003105E881F981EF93FF933196FA93EA93CC
:100A2C001EE01A9317EF91221FEB9122EFE3F0E0F7
:100A3C00B1E0BBBFB791BB2311F00E94225C1EE05A
:100A4C001F9318810F91011B102FFF91EF911083B1
:100A5C0023960C94A305153011F00C945705E881DE
:100A6C00F981EF93FF933196FA93EA931EE01A9370
:100A7C0017EF91221FEB9122E4E4F0E0B1E0BBBF51
:100A8C00B791BB2311F00E94225C1EE01F931881CA
:100A9C000F91011B102FFF91EF91108323960C9453
:100AAC00A305163011F00C947D05E881F981EF93C4
:100ABC00FF933196FA93EA931EE01A9317EF912263
:100ACC001FEB9122E9E4F0E0B1E0BBBFB791BB238F
:100ADC0011F00E94225C1EE01F9318810F91011BE4
:100AEC00102FFF91EF91108323960C94A3051730D0
:100AFC0011F00C94A305E881F981EF93FF933196E3
:100B0C00FA93EA931EE01A9317EF91221FEB9122AE
:100B1C00EEE4F0E0B1E0BBBFB791BB2311F00E9453
:100B2C00225C1EE01F9318810F91011B102FFF9167
:100B3C00EF91108323960C94A305FE013296319607
:100B4C001081193010E011F008F01FEF112311F48F
:100B5C000C94D605E881F981EF93FF933196FA93C3
:100B6C00EA931EE01A9317EF91221FEB9122EB816F
:100B7C00FC810E942A5CFE0135963196108150E072
:100B8C0040E0E0E20E94345C1EE01F9318810F915C
:100B9C00011B102FFF91EF91108323960C94FD05F0
:100BAC00E881F981EF93FF933196FA93EA931EE073
:100BBC001A9317EF91221FEB9122EB81FC810E947B
:100BCC002A5C10E30E94FE61FE013596319610817D
:100BDC0050E040E0E0E20E94345C1EE01F9318817C
:100BEC000F91011B102FFF91EF9110832396E88139
:100BFC00F981EF93FF933196FA93EA931EE01A93DF
:100C0C0017EF91221FEB9122EB81FC810E942A5C51
:100C1C001EE20E94FE611EE01F9318810F91011BC2
:100C2C00102FFF91EF9110832396FE01329632968E
:100C3C001081193010E011F008F01FEF112311F49E
:100C4C000C944E06E881F981EF93FF933196FA9359
:100C5C00EA931EE01A9317EF91221FEB9122EB817E
:100C6C00FC810E942A5CFE0135963296108150E080
:100C7C0040E0E0E20E94345C1EE01F9318810F916B
:100C8C00011B102FFF91EF91108323960C94750686
:100C9C00E881F981EF93FF933196FA93EA931EE082
:100CAC001A9317EF91221FEB9122EB81FC810E948A
:100CBC002A5C10E30E94FE61FE013596329610818B
:100CCC0050E040E0E0E20E94345C1EE01F9318818B
:100CDC000F91011B102FFF91EF9110832396E88148
:100CEC00F981EF93FF933196FA93EA931EE01A93EE
:100CFC0017EF91221FEB9122EB81FC810E942A5C61
:100D0C001EE20E94FE611EE01F9318810F91011BD1
:100D1C00102FFF91EF9110832396E881F981EF93C7
:100D2C00FF933196FA93EA931EE01A9317EF9122F0
:100D3C001FEB9122EB81FC810E942A5CFE0135960F
:100D4C003396108128E00E94376250E040E0E0E2E8
:100D5C000E94345C1EE01F9318810F91011B102F11
:100D6C00FF91EF9110832396E881F981EF93FF9324
:100D7C003196FA93EA931EE01A9317EF91221FEB28
:100D8C009122EB81FC810E942A5CFE013596339600
:100D9C00108150E040E0E0E20E94345C1EE01F93C2
:100DAC0018810F91011B102FFF91EF911083239647
:100DBC0008952497CF93DF93FE018F011A930A9322
:100DCC000E94C300DF91CF91112311F40C940307FF
:100DDC00CF93DF93FE01249724E030E0DE010E94E4
:100DEC00425B08851985F8011A930A930E949604B0
:100DFC00DF91CF911FEF0C94040710E00895239717
:100E0C00CF93DF93FE018F011A930A930E94630024
:100E1C00DF91CF91112311F40C942907CF93DF9319
:100E2C00FE01239723E030E0DE010E94425B0E813D
:100E3C001F81F8011A930A930E945603DF91CF91F8
:100E4C001FEF0C942A0710E008951881103011F050
:100E5C000C944B07F89418E697FC78941F9317E0C2
:100E6C001F93E89490F8E6E1F0E03F914F91A1E0F8
:100E7C00B0E060E00E94224E112311F40C9449075B
:100E8C001FEF0C94C8070C94C707113011F00C9489
:100E9C006A07F89418E697FC78941F9317E01F9351
:100EAC00E89490F8E6E1F0E03F914F91A1E0B0E0DA
:100EBC0060E10E94224E112311F40C9468071FEF7D
:100ECC000C94C8070C94C707123011F00C948907C6
:100EDC00F89418E697FC78941F9317E01F93E89406
:100EEC0090F8E6E1F0E03F914F91A1E0B0E061E1D4
:100EFC000E94224E112311F40C9487071FEF0C94BF
:100F0C00C8070C94C707133011F00C94A807F89479
:100F1C0018E697FC78941F9317E01F93E89490F8C9
:100F2C00E6E1F0E03F914F91A1E0B0E062E10E9478
:100F3C00224E112311F40C94A6071FEF0C94C80732
:100F4C000C94C707143011F00C94C707F89418E6EA
:100F5C0097FC78941F9317E01F93E89490F8E6E1C0
:100F6C00F0E03F914F91A1E0B0E063E10E94224E8E
:100F7C00112311F40C94C5071FEF0C94C8070C94A3
:100F8C00C70710E008951981173331F020F41030A1
:100F9C0010F0442701C041E010E009F41FEF1123C9
:100FAC0011F40C94F107F89418E697FC78941F93BD
:100FBC001981195F1F93E89490F8FE01A1E0B0E04D
:100FCC003F914F910E94224E112311F40C94F10782
:100FDC001FEF0C94F20710E008951A81173331F0CB
:100FEC0020F4113010F0442701C041E010E009F466
:100FFC001FEF112311F40C942908F89418E697FCB0
:10100C0078941F931A81195F312FE89490F84F91BF
:10101C00A0E0B0E00E94224E112311F40C94290898
:10102C00F89418E697FC78941F93E881F981A1E075
:10103C00B0E04F910E94104E112311F40C9429082A
:10104C001FEF0C942A0810E00895089509811A8165
:10105C00F80100935D0510935E05188110935F05F0
:10106C0011E11093600508952397FE01FA93EA931A
:10107C0010E01083EF93FF9310915F051150FF91D7
:10108C00EF911A931081088101171FEF08F01127B7
:10109C00112311F00C949008FE013496EF93FF93FA
:1010AC0000915D0510915E050F931F931B811F939B
:1010BC00109160050F910E945162012F11273F91F1
:1010CC002F91020F131FFF91EF9101931193FE01CA
:1010DC003696EF93FF93EC81FD813196BF91AF91E2
:1010EC00E89494F80E94355D10E009F41FEF112389
:1010FC0011F40C948708EC81FD81108123960C94DB
:10110C009208E981FA81108113951083112311F053
:10111C000C944908239610E008952197FE01FA9348
:10112C00EA9310E010831AE01A93108108810117DA
:10113C001FEF08F01127112311F00C94E608FE01A3
:10114C003496EF93FF93E2EAF4E0EF93FF931B8165
:10115C00012F1127A1E1B0E0E89495F80E946A6292
:10116C00FF91EF91E00FF11F3196BF91AF91E89491
:10117C0094F80E94355D10E009F41FEF112311F46F
:10118C000C94DD08E2EAF4E0EF93FF931B81012F4E
:10119C001127A1E1B0E0E89495F80E946A62FF91F2
:1011AC00EF91E00FF11F108123960C94E808E98170
:1011BC00FA81108113951083112311F00C949C0863
:1011CC00239610E00895279710E01E830E944D4E41
:1011DC001D831D81103310E008F01FEF1F931D813C
:1011EC0019331FEF10F009F011270F911023112361
:1011FC0011F40C942509CF93DF9318E0912A0BE797
:10120C001EE41A930A93FE01379610810E94FE6128
:10121C00DF91CF91FE013696108113951083FE015C
:10122C00EF93FF931E81FF91EF91012F1127E00F98
:10123C00F11FEF93FF931D81FF91EF9111931D818E
:10124C001D3010E009F41FEF112311F40C94EC087D
:10125C00FE01EF93FF931E81FF91EF911193FE011D
:10126C001FEB9122E89491F800E00E94655B102F2F
:10127C000895279710E01E830E944D4E1D831D81FB
:10128C00103310E008F01FEF1F931D8119331FEF6F
:10129C0010F009F011270F911023112311F40C9465
:1012AC007B09CF93DF9318E0912A0BE71EE41A9386
:1012BC000A93FE01379610810E94FE61DF91CF9157
:1012CC00FE013696108113951083FE01EF93FF9368
:1012DC001E81FF91EF91012F1127E00FF11FEF936A
:1012EC00FF931D81FF91EF9111931D811D3010E033
:1012FC0009F41FEF112311F40C944209FE01EF9332
:10130C00FF931E81FF91EF911193FE013196108195
:10131C00105324E00E9437621F93FE013296108115
:10132C0010530F91100F1E831E81089522970E9457
:10133C004D4E113618F01B3708F410521983CF9309
:10134C00DF9318E0912A0BE71EE41A930A93FE012F
:10135C00339610810E94FE61DF91CF911981193370
:10136C0010E011F008F01FEF112311F40C94C609D2
:10137C001981175300E10E94516218830C94CC0917
:10138C001981105300E10E94516218830E944D4E46
:10139C00113618F01B3708F410521983CF93DF93D2
:1013AC0018E0912A0BE71EE41A930A93FE01339678
:1013BC0010810E94FE61DF91CF911981193310E0E9
:1013CC0011F008F01FEF112311F40C94F609188199
:1013DC001F9319810F91100F175318830C94FD094B
:1013EC0018811F9319810F91100F105318831881B6
:1013FC000895249714E01B8310E000E01A830983FE
:10140C000E944D4E113618F01B3708F410521883F9
:10141C00CF93DF9318E0912A0BE71EE41A930A93FB
:10142C00FE01329610810E94FE61DF91CF91FE0188
:10143C00339610811A9510831881193310E011F02E
:10144C0008F01FEF112311F40C94450A09811A813D
:10145C000F931F931881012F1127075310400F93DF
:10146C001F931B8104E00E9451620E945A633F91BA
:10147C002F91020F131F1A8309830C945C0A0981A4
:10148C001A810F931F931881012F112700531040BD
:10149C000F931F931B8104E00E9451620E945A63B8
:1014AC003F912F91020F131F1A83098318811D304E
:1014BC0010E009F41FEF1F931B81103010E009F4AA
:1014CC001FEF0F91102B112311F40C94060A0981B4
:1014DC001A810895229710E019830E944D4E1883AB
:1014EC0018811D3010E009F41FEF1F9318811B3178
:1014FC0010E009F41FEF0F91102B112311F40C9431
:10150C008B0A0C94D40A0C94B00ACF93DF9318E096
:10151C00912A0BE71EE41A930A93FE01329610816E
:10152C000E94FE61DF91CF91FE01319610811395DF
:10153C001083EB81FC81EF93FF931981FF91EF9165
:10154C00012F1127E00FF11FEF93FF931881FF91EB
:10155C00EF91119318811D3010E009F41FEF1F93C8
:10156C0018811B3110E009F41FEF0F91102B1F9302
:10157C001881113110E009F41FEF0F91102B1F93FC
:10158C0019811F931A810F91011710E009F41FEFB5
:10159C000F91102B112311F40C94730AEB81FC8125
:1015AC00EF93FF931981FF91EF9111930895259774
:1015BC00F89410E597FC78941F930D811E81980187
:1015CC00689490F84F91A0E0B0E00E94224ECF9327
:1015DC00DF9318E0912A0BE71EE41A930A931DE09F
:1015EC000E94FE611AE00E94FE61DF91CF91FE0124
:1015FC003496FA93EA9310E010831FE01A9310814B
:10160C00088101171FEF08F01127112311F00C941A
:10161C00190CCF93DF9318E0912A0BE71EE41A9371
:10162C000A93F89410E097FC7894412F0E94505D37
:10163C00E3E5F0E0B1E0BBBFB791BB2311F00E9432
:10164C00225CDF91CF91CF93DF9318E0912A0BE7C7
:10165C001EE41A930A930A851B85D80120E031E019
:10166C00E89495F80E948C62102F412F0E94505DD7
:10167C000A851B85D80120E031E0E89495F80E949A
:10168C008C628F01507821F0019509F41A95109510
:10169C00102F412F0E94505DE6E5F0E0B1E0BBBF9A
:1016AC00B791BB2311F00E94225CDF91CF91FE0118
:1016BC003696FA93EA9310E010831FE01A93108188
:1016CC00088101171FEF08F01127112311F00C945A
:1016DC00950BF89410E597FC78941F93FE013896BF
:1016EC00A1E0B0E04F910E94104ECF93DF9318E031
:1016FC00912A0BE71EE41A930A931A85412F0E9434
:10170C00505D10E20E94FE61DF91CF91E981FA8178
:10171C00108113951083112311F00C94660B2396F2
:10172C00F89410E597FC78941F9308851985980117
:10173C00689490F84F91A0E0B0E00E94224EFE0118
:10174C003696FA93EA9310E010831FE01A931081F7
:10175C00088101171FEF08F01127112311F00C94C9
:10176C00F90BF89410E597FC78941F93FE013896CA
:10177C00A1E0B0E04F910E94104E1885103210E09D
:10178C0008F01FEF1F9318851F371FEF08F0112764
:10179C000F911023112311F40C94E30BCF93DF93CF
:1017AC0018E0912A0BE71EE41A930A931A850E94FB
:1017BC00FE61DF91CF910C94F00BCF93DF9318E087
:1017CC00912A0BE71EE41A930A931EE20E94FE6113
:1017DC00DF91CF91E981FA81108113951083112348
:1017EC0011F00C94AE0B2396CF93DF9318E0912A53
:1017FC000BE71EE41A930A931DE00E94FE611AE0A7
:10180C000E94FE61DF91CF9108851985005F1F4F03
:10181C0019870887E981FA811081139510831123A8
:10182C0011F00C94060B239608952197FE01FA9360
:10183C00EA9317E0108310E01A93108108810117C6
:10184C0010E011F008F01FEF112311F00C94710C43
:10185C001C811F931B81212F11E00E9437620F9175
:10186C001023103010E011F008F01FEF112311F4C9
:10187C000C94550CCF93DF9318E0912A0BE71EE4E0
:10188C001A930A93EAE5F0E0B1E0BBBFB791BB2332
:10189C0011F00E94225CDF91CF910C94680CCF93D5
:1018AC00DF9318E0912A0BE71EE41A930A93EDE5F7
:1018BC00F0E0B1E0BBBFB791BB2311F00E94225CFA
:1018CC00DF91CF91E981FA8110811A9510831F3F26
:1018DC0011F00C94240C239608952197FE01FA9391
:1018EC00EA9317E0108310E01A9310810881011716
:1018FC0010E011F008F01FEF112311F00C94C90C3B
:10190C001C811F931B81212F11E00E9437620F91C4
:10191C001023103010E011F008F01FEF112311F418
:10192C000C94AD0CCF93DF9318E0912A0BE71EE4D7
:10193C001A930A93E0E6F0E0B1E0BBBFB791BB238A
:10194C0011F00E94225CDF91CF910C94C00CCF93CC
:10195C00DF9318E0912A0BE71EE41A930A93E3E64F
:10196C00F0E0B1E0BBBFB791BB2311F00E94225C49
:10197C00DF91CF91E981FA8110811A9510831F3F75
:10198C0011F00C947C0C239608952197FE01FA9388
:10199C00EA9317E0108310E01A9310810881011765
:1019AC0010E011F008F01FEF112311F00C94480D0A
:1019BC001D811F931B81212F11E00E9437620F9113
:1019CC001023103010E011F008F01FEF112311F468
:1019DC000C94050DCF93DF9318E0912A0BE71EE4CE
:1019EC001A930A93E6E6F0E0B1E0BBBFB791BB23D4
:1019FC0011F00E94225CDF91CF910C943F0D1C8161
:101A0C001F931B81212F11E00E9437620F9110232D
:101A1C00103010E011F008F01FEF112311F40C94AA
:101A2C002C0DCF93DF9318E0912A0BE71EE41A9349
:101A3C000A93E9E6F0E0B1E0BBBFB791BB2311F02C
:101A4C000E94225CDF91CF910C943F0DCF93DF93DA
:101A5C0018E0912A0BE71EE41A930A93ECE6F0E0E7
:101A6C00B1E0BBBFB791BB2311F00E94225CDF91A8
:101A7C00CF91E981FA8110811A9510831F3F11F0E3
:101A8C000C94D40C23960895CF93DF9318E0912AED
:101A9C000BE71EE41A930A931DE00E94FE611AE004
:101AAC000E94FE61DF91CF91CF93DF9318E0912AD2
:101ABC000BE71EE41A930A93EFE6F0E0B1E0BBBF2C
:101ACC00B791BB2311F00E94225C1DE00E94FE61C5
:101ADC001AE00E94FE61DF91CF91CF93DF9318E063
:101AEC00912A0BE71EE41A930A93EAE7F0E0B1E0BF
:101AFC00BBBFB791BB2311F00E94225C1DE00E947A
:101B0C00FE611AE00E94FE61DF91CF91CF93DF93CB
:101B1C0018E0912A0BE71EE41A930A93EDEAF0E021
:101B2C00B1E0BBBFB791BB2311F00E94225C1DE05A
:101B3C000E94FE611AE00E94FE61DF91CF91CF936B
:101B4C00DF9318E0912A0BE71EE41A930A93E1ED58
:101B5C00F0E0B1E0BBBFB791BB2311F00E94225C57
:101B6C001DE00E94FE611AE00E94FE61DF91CF91A0
:101B7C00CF93DF9318E0912A0BE71EE41A930A9394
:101B8C00E5EFF0E0B1E0BBBFB791BB2311F00E94D1
:101B9C00225C1DE00E94FE611AE00E94FE61DF9152
:101BAC00CF91CF93DF9318E0912A0BE71EE41A93A1
:101BBC000A93E8E2F1E0B1E0BBBFB791BB2311F0AF
:101BCC000E94225C1DE00E94FE611AE00E94FE61F0
:101BDC00DF91CF91CF93DF9318E0912A0BE71EE4AE
:101BEC001A930A93E3E5F1E0B1E0BBBFB791BB23D5
:101BFC0011F00E94225C1DE00E94FE611AE00E941E
:101C0C00FE61DF91CF91CF93DF9318E0912A0BE720
:101C1C001EE41A930A93E2E7F1E0B1E0BBBFB7917F
:101C2C00BB2311F00E94225C1DE00E94FE611AE0B1
:101C3C000E94FE61DF91CF91CF93DF9318E0912A40
:101C4C000BE71EE41A930A93E6E9F1E0B1E0BBBF9F
:101C5C00B791BB2311F00E94225C1DE00E94FE6133
:101C6C001AE00E94FE61DF91CF91CF93DF9318E0D1
:101C7C00912A0BE71EE41A930A93E6EBF1E0B1E02C
:101C8C00BBBFB791BB2311F00E94225C1DE00E94E8
:101C9C00FE611AE00E94FE61DF91CF91CF93DF933A
:101CAC0018E0912A0BE71EE41A930A93E1EDF1E098
:101CBC00B1E0BBBFB791BB2311F00E94225C1DE0C9
:101CCC000E94FE611AE00E94FE61DF91CF91CF93DA
:101CDC00DF9318E0912A0BE71EE41A930A93ECEEBB
:101CEC00F1E0B1E0BBBFB791BB2311F00E94225CC5
:101CFC001DE00E94FE611AE00E94FE61DF91CF910F
:101D0C00CF93DF9318E0912A0BE71EE41A930A9302
:101D1C00E8E1F2E0B1E0BBBFB791BB2311F00E9448
:101D2C00225C1DE00E94FE611AE00E94FE61DF91C0
:101D3C00CF91CF93DF9318E0912A0BE71EE41A930F
:101D4C000A93E8E3F2E0B1E0BBBFB791BB2311F01B
:101D5C000E94225C1DE00E94FE611AE00E94FE615E
:101D6C00DF91CF91089523971B81103010E009F477
:101D7C001FEF112311F40C94DE0EFE01EF93FF9371
:101D8C003196FA93EA9312E01A9317EF91221FEB14
:101D9C00912211E30E94FE6112E01F9318810F91B2
:101DAC00011B102FFF91EF91108323960C94F70ECB
:101DBC00FE01EF93FF933196FA93EA9312E01A9394
:101DCC0017EF91221FEB912212E30E94FE6112E0A9
:101DDC001F9318810F91011B102FFF91EF9110830E
:101DEC002396CF93DF9318E0912A0BE71EE41A9306
:101DFC000A931DE00E94FE611AE00E94FE61DF91D1
:101E0C00CF91CF93DF9318E0912A0BE71EE41A933E
:101E1C000A93ECE5F2E0B1E0BBBFB791BB2311F044
:101E2C000E94225C1DE00E94FE611AE00E94FE618D
:101E3C00DF91CF91CF93DF9318E0912A0BE71EE44B
:101E4C001A930A93E7E9F2E0B1E0BBBFB791BB2369
:101E5C0011F00E94225C1DE00E94FE611AE00E94BB
:101E6C00FE61DF91CF91CF93DF9318E0912A0BE7BE
:101E7C001EE41A930A93E2EDF2E0B1E0BBBFB79116
:101E8C00BB2311F00E94225C1DE00E94FE611AE04F
:101E9C000E94FE61DF91CF91CF93DF9318E0912ADE
:101EAC000BE71EE41A930A93ECE5F2E0B1E0BBBF3A
:101EBC00B791BB2311F00E94225C1DE00E94FE61D1
:101ECC001AE00E94FE61DF91CF91CF93DF9318E06F
:101EDC00912A0BE71EE41A930A93EDE0F3E0B1E0CC
:101EEC00BBBFB791BB2311F00E94225CFE0132965E
:101EFC000E942A5CE6E3F3E0B1E0BBBFB791BB23E1
:101F0C0011F00E94225C1DE00E94FE611AE00E940A
:101F1C00FE61DF91CF9108952197CF93DF9318E065
:101F2C00912A0BE71EE41A930A931DE00E94FE61AE
:101F3C001AE00E94FE61DF91CF91CF93DF9318E0FE
:101F4C00912A0BE71EE41A930A93EAE3F3E0B1E05B
:101F5C00BBBFB791BB2311F00E94225C10919D0076
:101F6C00412F0E945D5D1DE00E94FE611AE00E94FF
:101F7C00FE61DF91CF91CF93DF9318E0912A0BE7AD
:101F8C001EE41A930A93E4E4F3E0B1E0BBBFB7910B
:101F9C00BB2311F00E94225C10919C00412F0E94E7
:101FAC005D5D1DE00E94FE611AE00E94FE61DF9102
:101FBC00CF91CF93DF9318E0912A0BE71EE41A938D
:101FCC000A93EEE4F3E0B1E0BBBFB791BB2311F091
:101FDC000E94225C10919B00412F0E945D5D1DE0D0
:101FEC000E94FE611AE00E94FE61DF91CF91CF93B7
:101FFC00DF9318E0912A0BE71EE41A930A93E8E5A5
:10200C00F3E0B1E0BBBFB791BB2311F00E94225C9F
:10201C0010919B00412F0E945D5D1DE00E94FE61AE
:10202C001AE00E94FE61DF91CF91CF93DF9318E00D
:10203C00912A0BE71EE41A930A93E2E6F3E0B1E06F
:10204C00BBBFB791BB2311F00E94225C10919A0088
:10205C00412F0E945D5D1DE00E94FE611AE00E940E
:10206C00FE61DF91CF91CF93DF9318E0912A0BE7BC
:10207C001EE41A930A93ECE6F3E0B1E0BBBFB79110
:10208C00BB2311F00E94225C10919A00412F0E94F8
:10209C005D5D1DE00E94FE611AE00E94FE61DF9111
:1020AC00CF91CF93DF9318E0912A0BE71EE41A939C
:1020BC000A93E6E7F3E0B1E0BBBFB791BB2311F0A5
:1020CC000E94225C10919900412F0E945D5D1DE0E1
:1020DC000E94FE611AE00E94FE61DF91CF91CF93C6
:1020EC00DF9318E0912A0BE71EE41A930A93E0E8B9
:1020FC00F3E0B1E0BBBFB791BB2311F00E94225CAF
:10210C0010919900412F0E945D5D1DE00E94FE61BF
:10211C001AE00E94FE61DF91CF91CF93DF9318E01C
:10212C00912A0BE71EE41A930A93EAE8F3E0B1E074
:10213C00BBBFB791BB2311F00E94225C1091980099
:10214C00412F0E945D5D1DE00E94FE611AE00E941D
:10215C00FE61DF91CF91CF93DF9318E0912A0BE7CB
:10216C001EE41A930A93E4E9F3E0B1E0BBBFB79124
:10217C00BB2311F00E94225C10919500412F0E940C
:10218C005D5D1DE00E94FE611AE00E94FE61DF9120
:10219C00CF91CF93DF9318E0912A0BE71EE41A93AB
:1021AC000A93EEE9F3E0B1E0BBBFB791BB2311F0AA
:1021BC000E94225C10919500412F0E945D5D1DE0F4
:1021CC000E94FE611AE00E94FE61DF91CF91CF93D5
:1021DC00DF9318E0912A0BE71EE41A930A93E8EABE
:1021EC00F3E0B1E0BBBFB791BB2311F00E94225CBE
:1021FC001DE00E94FE611AE00E94FE61DF91CF910A
:10220C000E944D4E1883CF93DF9318E0912A0BE771
:10221C001EE41A930A93E9EBF3E0B1E0BBBFB7916C
:10222C00BB2311F00E94225C10919000412F0E9460
:10223C005D5D1DE00E94FE611AE00E94FE61DF916F
:10224C00CF91CF93DF9318E0912A0BE71EE41A93FA
:10225C000A93E3ECF3E0B1E0BBBFB791BB2311F001
:10226C000E94225C10919000412F0E945D5D1DE048
:10227C000E94FE611AE00E94FE61DF91CF91CF9324
:10228C00DF9318E0912A0BE71EE41A930A93EDEC06
:10229C00F3E0B1E0BBBFB791BB2311F00E94225C0D
:1022AC0010918C00412F0E945D5D1DE00E94FE612B
:1022BC001AE00E94FE61DF91CF91CF93DF9318E07B
:1022CC00912A0BE71EE41A930A93E7EDF3E0B1E0D1
:1022DC00BBBFB791BB2311F00E94225C10918B0005
:1022EC00412F0E945D5D1DE00E94FE611AE00E947C
:1022FC00FE61DF91CF91CF93DF9318E0912A0BE72A
:10230C001EE41A930A93E1EEF3E0B1E0BBBFB79180
:10231C00BB2311F00E94225C10918A00412F0E9475
:10232C005D5D1DE00E94FE611AE00E94FE61DF917E
:10233C00CF91CF93DF9318E0912A0BE71EE41A9309
:10234C000A93EBEEF3E0B1E0BBBFB791BB2311F006
:10235C000E94225C10918900412F0E945D5D1DE05E
:10236C000E94FE611AE00E94FE61DF91CF91CF9333
:10237C00DF9318E0912A0BE71EE41A930A93E5EF1A
:10238C00F3E0B1E0BBBFB791BB2311F00E94225C1C
:10239C0010918800412F0E945D5D1DE00E94FE613E
:1023AC001AE00E94FE61DF91CF91CF93DF9318E08A
:1023BC00912A0BE71EE41A930A93EFEFF3E0B1E0D6
:1023CC00BBBFB791BB2311F00E94225C1091870018
:1023DC00412F0E945D5D1DE00E94FE611AE00E948B
:1023EC00FE61DF91CF91CF93DF9318E0912A0BE739
:1023FC001EE41A930A93E9E0F4E0B1E0BBBFB79195
:10240C00BB2311F00E94225C10918600412F0E9488
:10241C005D5D1DE00E94FE611AE00E94FE61DF918D
:10242C00CF91CF93DF9318E0912A0BE71EE41A9318
:10243C000A93E3E1F4E0B1E0BBBFB791BB2311F029
:10244C000E94225C10918500412F0E945D5D1DE071
:10245C000E94FE611AE00E94FE61DF91CF91CF9342
:10246C00DF9318E0912A0BE71EE41A930A93E8EA2B
:10247C00F3E0B1E0BBBFB791BB2311F00E94225C2B
:10248C001DE00E94FE611AE00E94FE61DF91CF9177
:10249C000E944D4E1883CF93DF9318E0912A0BE7DF
:1024AC001EE41A930A93EDE1F4E0B1E0BBBFB791DF
:1024BC00BB2311F00E94225C10918400412F0E94DA
:1024CC005D5D1DE00E94FE611AE00E94FE61DF91DD
:1024DC00CF91CF93DF9318E0912A0BE71EE41A9368
:1024EC000A93E7E2F4E0B1E0BBBFB791BB2311F074
:1024FC000E94225C10918300412F0E945D5D1DE0C3
:10250C000E94FE611AE00E94FE61DF91CF91CF9391
:10251C00DF9318E0912A0BE71EE41A930A93E1E388
:10252C00F4E0B1E0BBBFB791BB2311F00E94225C79
:10253C0010918200412F0E945D5D1DE00E94FE61A2
:10254C001AE00E94FE61DF91CF91CF93DF9318E0E8
:10255C00912A0BE71EE41A930A93EBE3F4E0B1E043
:10256C00BBBFB791BB2311F00E94225C109181007C
:10257C00412F0E945D5D1DE00E94FE611AE00E94E9
:10258C00FE61DF91CF91CF93DF9318E0912A0BE797
:10259C001EE41A930A93E5E4F4E0B1E0BBBFB791F3
:1025AC00BB2311F00E94225C10918000412F0E94ED
:1025BC005D5D1DE00E94FE611AE00E94FE61DF91EC
:1025CC00CF91CF93DF9318E0912A0BE71EE41A9377
:1025DC000A93EFE4F4E0B1E0BBBFB791BB2311F079
:1025EC000E94225C10917D00412F0E945D5D1DE0D8
:1025FC000E94FE611AE00E94FE61DF91CF91CF93A1
:10260C00DF9318E0912A0BE71EE41A930A93E9E58D
:10261C00F4E0B1E0BBBFB791BB2311F00E94225C88
:10262C0010917C00412F0E945D5D1DE00E94FE61B7
:10263C001AE00E94FE61DF91CF91CF93DF9318E0F7
:10264C00912A0BE71EE41A930A93E3E6F4E0B1E057
:10265C00BBBFB791BB2311F00E94225C10917A0092
:10266C00412F0E945D5D1DE00E94FE611AE00E94F8
:10267C00FE61DF91CF91CF93DF9318E0912A0BE7A6
:10268C001EE41A930A93EDE6F4E0B1E0BBBFB791F8
:10269C00BB2311F00E94225C10917900412F0E9403
:1026AC005D5D1DE00E94FE611AE00E94FE61DF91FB
:1026BC00CF91CF93DF9318E0912A0BE71EE41A9386
:1026CC000A93E7E7F4E0B1E0BBBFB791BB2311F08D
:1026DC000E94225C10917800412F0E945D5D1DE0EC
:1026EC000E94FE611AE00E94FE61DF91CF91CF93B0
:1026FC00DF9318E0912A0BE71EE41A930A93E8EA99
:10270C00F3E0B1E0BBBFB791BB2311F00E94225C98
:10271C001DE00E94FE611AE00E94FE61DF91CF91E4
:10272C000E944D4E1883CF93DF9318E0912A0BE74C
:10273C001EE41A930A93E1E8F4E0B1E0BBBFB79151
:10274C00BB2311F00E94225C10917400412F0E9457
:10275C005D5D1DE00E94FE611AE00E94FE61DF914A
:10276C00CF91CF93DF9318E0912A0BE71EE41A93D5
:10277C000A93EBE8F4E0B1E0BBBFB791BB2311F0D7
:10278C000E94225C10917300412F0E945D5D1DE040
:10279C000E94FE611AE00E94FE61DF91CF91CF93FF
:1027AC00DF9318E0912A0BE71EE41A930A93E5E9EC
:1027BC00F4E0B1E0BBBFB791BB2311F00E94225CE7
:1027CC0010917200412F0E945D5D1DE00E94FE6120
:1027DC001AE00E94FE61DF91CF91CF93DF9318E056
:1027EC00912A0BE71EE41A930A93EFE9F4E0B1E0A7
:1027FC00BBBFB791BB2311F00E94225C10917100FA
:10280C00412F0E945D5D1DE00E94FE611AE00E9456
:10281C00FE61DF91CF91CF93DF9318E0912A0BE704
:10282C001EE41A930A93E9EAF4E0B1E0BBBFB79156
:10283C00BB2311F00E94225C10917000412F0E946A
:10284C005D5D1DE00E94FE611AE00E94FE61DF9159
:10285C00CF91CF93DF9318E0912A0BE71EE41A93E4
:10286C000A93E3EBF4E0B1E0BBBFB791BB2311F0EB
:10287C000E94225C10916F00412F0E945D5D1DE053
:10288C000E94FE611AE00E94FE61DF91CF91CF930E
:10289C00DF9318E0912A0BE71EE41A930A93EDEBF1
:1028AC00F4E0B1E0BBBFB791BB2311F00E94225CF6
:1028BC0010916D00412F0E945D5D1DE00E94FE6134
:1028CC001AE00E94FE61DF91CF91CF93DF9318E065
:1028DC00912A0BE71EE41A930A93E7ECF4E0B1E0BB
:1028EC00BBBFB791BB2311F00E94225C10916C000E
:1028FC00412F0E945D5D1DE00E94FE611AE00E9466
:10290C00FE61DF91CF91CF93DF9318E0912A0BE713
:10291C001EE41A930A93E1EDF4E0B1E0BBBFB7916A
:10292C00BB2311F00E94225C10916A00412F0E947F
:10293C005D5D1DE00E94FE611AE00E94FE61DF9168
:10294C00CF91CF93DF9318E0912A0BE71EE41A93F3
:10295C000A93EBEDF4E0B1E0BBBFB791BB2311F0F0
:10296C000E94225C10916800412F0E945D5D1DE069
:10297C000E94FE611AE00E94FE61DF91CF91CF931D
:10298C00DF9318E0912A0BE71EE41A930A93E8EA06
:10299C00F3E0B1E0BBBFB791BB2311F00E94225C06
:1029AC001DE00E94FE611AE00E94FE61DF91CF9152
:1029BC000E944D4E1883CF93DF9318E0912A0BE7BA
:1029CC001EE41A930A93E5EEF4E0B1E0BBBFB791B5
:1029DC00BB2311F00E94225C10916800412F0E94D1
:1029EC005D5D1DE00E94FE611AE00E94FE61DF91B8
:1029FC00CF91CF93DF9318E0912A0BE71EE41A9343
:102A0C000A93EFEEF4E0B1E0BBBFB791BB2311F03A
:102A1C000E94225C10916500412F0E945D5D1DE0BB
:102A2C000E94FE611AE00E94FE61DF91CF91CF936C
:102A3C00DF9318E0912A0BE71EE41A930A93E9EF4F
:102A4C00F4E0B1E0BBBFB791BB2311F00E94225C54
:102A5C0010916400412F0E945D5D1DE00E94FE619B
:102A6C001AE00E94FE61DF91CF91CF93DF9318E0C3
:102A7C00912A0BE71EE41A930A93E3E0F5E0B1E028
:102A8C00BBBFB791BB2311F00E94225C1091630075
:102A9C00412F0E945D5D1DE00E94FE611AE00E94C4
:102AAC00FE61DF91CF91CF93DF9318E0912A0BE772
:102ABC001EE41A930A93EDE0F5E0B1E0BBBFB791C9
:102ACC00BB2311F00E94225C10916200412F0E94E6
:102ADC005D5D1DE00E94FE611AE00E94FE61DF91C7
:102AEC00CF91CF93DF9318E0912A0BE71EE41A9352
:102AFC000A93E7E1F5E0B1E0BBBFB791BB2311F05E
:102B0C000E94225C10916100412F0E945D5D1DE0CE
:102B1C000E94FE611AE00E94FE61DF91CF91CF937B
:102B2C00DF9318E0912A0BE71EE41A930A93E1E273
:102B3C00F5E0B1E0BBBFB791BB2311F00E94225C62
:102B4C001FB7412F0E945D5D1DE00E94FE611AE0DF
:102B5C000E94FE61DF91CF91CF93DF9318E0912A11
:102B6C000BE71EE41A930A93EBE2F5E0B1E0BBBF6E
:102B7C00B791BB2311F00E94225C1EB7412F0E941B
:102B8C005D5D1DE00E94FE611AE00E94FE61DF9116
:102B9C00CF91CF93DF9318E0912A0BE71EE41A93A1
:102BAC000A93E5E3F5E0B1E0BBBFB791BB2311F0AD
:102BBC000E94225C1DB7412F0E945D5D1DE00E94AA
:102BCC00FE611AE00E94FE61DF91CF91CF93DF93FB
:102BDC0018E0912A0BE71EE41A930A93EFE3F5E051
:102BEC00B1E0BBBFB791BB2311F00E94225C1CB7B4
:102BFC00412F0E945D5D1DE00E94FE611AE00E9463
:102C0C00FE61DF91CF91CF93DF9318E0912A0BE710
:102C1C001EE41A930A93E8EAF3E0B1E0BBBFB79164
:102C2C00BB2311F00E94225C1DE00E94FE611AE0A1
:102C3C000E94FE61DF91CF910E944D4E1883CF937D
:102C4C00DF9318E0912A0BE71EE41A930A93E9E448
:102C5C00F5E0B1E0BBBFB791BB2311F00E94225C41
:102C6C001BB7412F0E945D5D1DE00E94FE611AE0C2
:102C7C000E94FE61DF91CF91CF93DF9318E0912AF0
:102C8C000BE71EE41A930A93E3E5F5E0B1E0BBBF52
:102C9C00B791BB2311F00E94225C1AB7412F0E94FE
:102CAC005D5D1DE00E94FE611AE00E94FE61DF91F5
:102CBC00CF91CF93DF9318E0912A0BE71EE41A9380
:102CCC000A93EDE5F5E0B1E0BBBFB791BB2311F082
:102CDC000E94225C1AB7412F0E945D5D1DE00E948C
:102CEC00FE611AE00E94FE61DF91CF91CF93DF93DA
:102CFC0018E0912A0BE71EE41A930A93E7E6F5E035
:102D0C00B1E0BBBFB791BB2311F00E94225C19B795
:102D1C00412F0E945D5D1DE00E94FE611AE00E9441
:102D2C00FE61DF91CF91CF93DF9318E0912A0BE7EF
:102D3C001EE41A930A93E1E7F5E0B1E0BBBFB7914B
:102D4C00BB2311F00E94225C18B7412F0E945D5DDD
:102D5C001DE00E94FE611AE00E94FE61DF91CF919E
:102D6C00CF93DF9318E0912A0BE71EE41A930A9392
:102D7C00EBE7F5E0B1E0BBBFB791BB2311F00E94CC
:102D8C00225C17B7412F0E945D5D1DE00E94FE6121
:102D9C001AE00E94FE61DF91CF91CF93DF9318E090
:102DAC00912A0BE71EE41A930A93E5E8F5E0B1E0EB
:102DBC00BBBFB791BB2311F00E94225C16B7412F09
:102DCC000E945D5D1DE00E94FE611AE00E94FE61A2
:102DDC00DF91CF91CF93DF9318E0912A0BE71EE49C
:102DEC001A930A93EFE8F5E0B1E0BBBFB791BB23B0
:102DFC0011F00E94225C15B7412F0E945D5D1DE011
:102E0C000E94FE611AE00E94FE61DF91CF91CF9388
:102E1C00DF9318E0912A0BE71EE41A930A93E9E971
:102E2C00F5E0B1E0BBBFB791BB2311F00E94225C6F
:102E3C0014B7412F0E945D5D1DE00E94FE611AE0F7
:102E4C000E94FE61DF91CF91CF93DF9318E0912A1E
:102E5C000BE71EE41A930A93E3EAF5E0B1E0BBBF7B
:102E6C00B791BB2311F00E94225C13B7412F0E9433
:102E7C005D5D1DE00E94FE611AE00E94FE61DF9123
:102E8C00CF91CF93DF9318E0912A0BE71EE41A93AE
:102E9C000A93E8EAF3E0B1E0BBBFB791BB2311F0B2
:102EAC000E94225C1DE00E94FE611AE00E94FE61FD
:102EBC00DF91CF910E944D4E1883CF93DF9318E092
:102ECC00912A0BE71EE41A930A93EDEAF5E0B1E0C0
:102EDC00BBBFB791BB2311F00E94225C12B7412FEC
:102EEC000E945D5D1DE00E94FE611AE00E94FE6181
:102EFC00DF91CF91CF93DF9318E0912A0BE71EE47B
:102F0C001A930A93E7EBF5E0B1E0BBBFB791BB2393
:102F1C0011F00E94225C11B7412F0E945D5D1DE0F3
:102F2C000E94FE611AE00E94FE61DF91CF91CF9367
:102F3C00DF9318E0912A0BE71EE41A930A93E1EC55
:102F4C00F5E0B1E0BBBFB791BB2311F00E94225C4E
:102F5C0010B7412F0E945D5D1DE00E94FE611AE0DA
:102F6C000E94FE61DF91CF91CF93DF9318E0912AFD
:102F7C000BE71EE41A930A93EBECF5E0B1E0BBBF50
:102F8C00B791BB2311F00E94225C1FB5412F0E9408
:102F9C005D5D1DE00E94FE611AE00E94FE61DF9102
:102FAC00CF91CF93DF9318E0912A0BE71EE41A938D
:102FBC000A93E5EDF5E0B1E0BBBFB791BB2311F08F
:102FCC000E94225C1EB5412F0E945D5D1DE00E9497
:102FDC00FE611AE00E94FE61DF91CF91CF93DF93E7
:102FEC0018E0912A0BE71EE41A930A93EFEDF5E033
:102FFC00B1E0BBBFB791BB2311F00E94225C1DB5A1
:10300C00412F0E945D5D1DE00E94FE611AE00E944E
:10301C00FE61DF91CF91CF93DF9318E0912A0BE7FC
:10302C001EE41A930A93E9EEF5E0B1E0BBBFB79149
:10303C00BB2311F00E94225C1CB5412F0E945D5DE8
:10304C001DE00E94FE611AE00E94FE61DF91CF91AB
:10305C00CF93DF9318E0912A0BE71EE41A930A939F
:10306C00E3EFF5E0B1E0BBBFB791BB2311F00E94D9
:10307C00225C1BB5412F0E945D5D1DE00E94FE612C
:10308C001AE00E94FE61DF91CF91CF93DF9318E09D
:10309C00912A0BE71EE41A930A93EDEFF5E0B1E0E9
:1030AC00BBBFB791BB2311F00E94225C1AB5412F14
:1030BC000E945D5D1DE00E94FE611AE00E94FE61AF
:1030CC00DF91CF91CF93DF9318E0912A0BE71EE4A9
:1030DC001A930A93E7E0F6E0B1E0BBBFB791BB23CC
:1030EC0011F00E94225C19B5412F0E945D5D1DE01C
:1030FC000E94FE611AE00E94FE61DF91CF91CF9396
:10310C00DF9318E0912A0BE71EE41A930A93E8EA7E
:10311C00F3E0B1E0BBBFB791BB2311F00E94225C7E
:10312C001DE00E94FE611AE00E94FE61DF91CF91CA
:10313C000E944D4E1883CF93DF9318E0912A0BE732
:10314C001EE41A930A93E1E1F6E0B1E0BBBFB7913C
:10315C00BB2311F00E94225C18B5412F0E945D5DCB
:10316C001DE00E94FE611AE00E94FE61DF91CF918A
:10317C00CF93DF9318E0912A0BE71EE41A930A937E
:10318C00EBE1F6E0B1E0BBBFB791BB2311F00E94BD
:10319C00225C17B5412F0E945D5D1DE00E94FE610F
:1031AC001AE00E94FE61DF91CF91CF93DF9318E07C
:1031BC00912A0BE71EE41A930A93E5E2F6E0B1E0DC
:1031CC00BBBFB791BB2311F00E94225C16B5412FF7
:1031DC000E945D5D1DE00E94FE611AE00E94FE618E
:1031EC00DF91CF91CF93DF9318E0912A0BE71EE488
:1031FC001A930A93EFE2F6E0B1E0BBBFB791BB23A1
:10320C0011F00E94225C15B5412F0E945D5D1DE0FE
:10321C000E94FE611AE00E94FE61DF91CF91CF9374
:10322C00DF9318E0912A0BE71EE41A930A93E9E363
:10323C00F6E0B1E0BBBFB791BB2311F00E94225C5A
:10324C0014B5412F0E945D5D1DE00E94FE611AE0E5
:10325C000E94FE61DF91CF91CF93DF9318E0912A0A
:10326C000BE71EE41A930A93E3E4F6E0B1E0BBBF6C
:10327C00B791BB2311F00E94225C13B5412F0E9421
:10328C005D5D1DE00E94FE611AE00E94FE61DF910F
:10329C00CF91CF93DF9318E0912A0BE71EE41A939A
:1032AC000A93EDE4F6E0B1E0BBBFB791BB2311F09C
:1032BC000E94225C12B5412F0E945D5D1DE00E94B0
:1032CC00FE611AE00E94FE61DF91CF91CF93DF93F4
:1032DC0018E0912A0BE71EE41A930A93E7E5F6E04F
:1032EC00B1E0BBBFB791BB2311F00E94225C11B5BA
:1032FC00412F0E945D5D1DE00E94FE611AE00E945C
:10330C00FE61DF91CF91CF93DF9318E0912A0BE709
:10331C001EE41A930A93E1E6F6E0B1E0BBBFB79165
:10332C00BB2311F00E94225C1FB3412F0E945D5DF4
:10333C001DE00E94FE611AE00E94FE61DF91CF91B8
:10334C00CF93DF9318E0912A0BE71EE41A930A93AC
:10335C00EBE6F6E0B1E0BBBFB791BB2311F00E94E6
:10336C00225C1EB3412F0E945D5D1DE00E94FE6138
:10337C001AE00E94FE61DF91CF91CF93DF9318E0AA
:10338C00912A0BE71EE41A930A93E8EAF3E0B1E002
:10339C00BBBFB791BB2311F00E94225C1DE00E94C1
:1033AC00FE611AE00E94FE61DF91CF910E944D4EAA
:1033BC001883CF93DF9318E0912A0BE71EE41A933E
:1033CC000A93E5E7F6E0B1E0BBBFB791BB2311F080
:1033DC000E94225C1DB3412F0E945D5D1DE00E9486
:1033EC00FE611AE00E94FE61DF91CF91CF93DF93D3
:1033FC0018E0912A0BE71EE41A930A93EFE7F6E024
:10340C00B1E0BBBFB791BB2311F00E94225C1CB38F
:10341C00412F0E945D5D1DE00E94FE611AE00E943A
:10342C00FE61DF91CF91CF93DF9318E0912A0BE7E8
:10343C001EE41A930A93E9E8F6E0B1E0BBBFB7913A
:10344C00BB2311F00E94225C1BB3412F0E945D5DD7
:10345C001DE00E94FE611AE00E94FE61DF91CF9197
:10346C00CF93DF9318E0912A0BE71EE41A930A938B
:10347C00E3E9F6E0B1E0BBBFB791BB2311F00E94CA
:10348C00225C1AB3412F0E945D5D1DE00E94FE611B
:10349C001AE00E94FE61DF91CF91CF93DF9318E089
:1034AC00912A0BE71EE41A930A93EDE9F6E0B1E0DA
:1034BC00BBBFB791BB2311F00E94225C19B3412F03
:1034CC000E945D5D1DE00E94FE611AE00E94FE619B
:1034DC00DF91CF91CF93DF9318E0912A0BE71EE495
:1034EC001A930A93E7EAF6E0B1E0BBBFB791BB23AE
:1034FC0011F00E94225C18B3412F0E945D5D1DE00B
:10350C000E94FE611AE00E94FE61DF91CF91CF9381
:10351C00DF9318E0912A0BE71EE41A930A93E1EB70
:10352C00F6E0B1E0BBBFB791BB2311F00E94225C67
:10353C0017B3412F0E945D5D1DE00E94FE611AE0F1
:10354C000E94FE61DF91CF91CF93DF9318E0912A17
:10355C000BE71EE41A930A93EBEBF6E0B1E0BBBF6A
:10356C00B791BB2311F00E94225C16B3412F0E942D
:10357C005D5D1DE00E94FE611AE00E94FE61DF911C
:10358C00CF91CF93DF9318E0912A0BE71EE41A93A7
:10359C000A93E5ECF6E0B1E0BBBFB791BB2311F0A9
:1035AC000E94225C15B3412F0E945D5D1DE00E94BC
:1035BC00FE611AE00E94FE61DF91CF91CF93DF9301
:1035CC0018E0912A0BE71EE41A930A93EFECF6E04D
:1035DC00B1E0BBBFB791BB2311F00E94225C14B3C6
:1035EC00412F0E945D5D1DE00E94FE611AE00E9469
:1035FC00FE61DF91CF91CF93DF9318E0912A0BE717
:10360C001EE41A930A93E8EAF3E0B1E0BBBFB7916A
:10361C00BB2311F00E94225C1DE00E94FE611AE0A7
:10362C000E94FE61DF91CF910E944D4E1883CF9383
:10363C00DF9318E0912A0BE71EE41A930A93E9ED45
:10364C00F6E0B1E0BBBFB791BB2311F00E94225C46
:10365C0013B3412F0E945D5D1DE00E94FE611AE0D4
:10366C000E94FE61DF91CF91CF93DF9318E0912AF6
:10367C000BE71EE41A930A93E3EEF6E0B1E0BBBF4E
:10368C00B791BB2311F00E94225C12B3412F0E9410
:10369C005D5D1DE00E94FE611AE00E94FE61DF91FB
:1036AC00CF91CF93DF9318E0912A0BE71EE41A9386
:1036BC000A93EDEEF6E0B1E0BBBFB791BB2311F07E
:1036CC000E94225C11B3412F0E945D5D1DE00E949F
:1036DC00FE611AE00E94FE61DF91CF91CF93DF93E0
:1036EC0018E0912A0BE71EE41A930A93E7EFF6E031
:1036FC00B1E0BBBFB791BB2311F00E94225C10B3A9
:10370C00412F0E945D5D1DE00E94FE611AE00E9447
:10371C00FE61DF91CF91CF93DF9318E0912A0BE7F5
:10372C001EE41A930A93E1E0F7E0B1E0BBBFB79156
:10373C00BB2311F00E94225C1FB1412F0E945D5DE2
:10374C001DE00E94FE611AE00E94FE61DF91CF91A4
:10375C00CF93DF9318E0912A0BE71EE41A930A9398
:10376C00EBE0F7E0B1E0BBBFB791BB2311F00E94D7
:10377C00225C1EB1412F0E945D5D1DE00E94FE6126
:10378C001AE00E94FE61DF91CF91CF93DF9318E096
:10379C00912A0BE71EE41A930A93E5E1F7E0B1E0F6
:1037AC00BBBFB791BB2311F00E94225C1DB1412F0E
:1037BC000E945D5D1DE00E94FE611AE00E94FE61A8
:1037CC00DF91CF91CF93DF9318E0912A0BE71EE4A2
:1037DC001A930A93EFE1F7E0B1E0BBBFB791BB23BB
:1037EC0011F00E94225C1CB1412F0E945D5D1DE016
:1037FC000E94FE611AE00E94FE61DF91CF91CF938F
:10380C00DF9318E0912A0BE71EE41A930A93E9E27E
:10381C00F7E0B1E0BBBFB791BB2311F00E94225C73
:10382C001BB1412F0E945D5D1DE00E94FE611AE0FC
:10383C000E94FE61DF91CF91CF93DF9318E0912A24
:10384C000BE71EE41A930A93E3E3F7E0B1E0BBBF86
:10385C00B791BB2311F00E94225C1AB1412F0E9438
:10386C005D5D1DE00E94FE611AE00E94FE61DF9129
:10387C00CF91CF93DF9318E0912A0BE71EE41A93B4
:10388C000A93E8EAF3E0B1E0BBBFB791BB2311F0B8
:10389C000E94225C1DE00E94FE611AE00E94FE6103
:1038AC00DF91CF910E944D4E1883CF93DF9318E098
:1038BC00912A0BE71EE41A930A93EDE3F7E0B1E0CB
:1038CC00BBBFB791BB2311F00E94225C19B1412FF1
:1038DC000E945D5D1DE00E94FE611AE00E94FE6187
:1038EC00DF91CF91CF93DF9318E0912A0BE71EE481
:1038FC001A930A93E7E4F7E0B1E0BBBFB791BB239F
:10390C0011F00E94225C19B1412F0E945D5D1DE0F7
:10391C000E94FE611AE00E94FE61DF91CF91CF936D
:10392C00DF9318E0912A0BE71EE41A930A93E1E562
:10393C00F7E0B1E0BBBFB791BB2311F00E94225C52
:10394C0018B1412F0E945D5D1DE00E94FE611AE0DE
:10395C000E94FE61DF91CF91CF93DF9318E0912A03
:10396C000BE71EE41A930A93EBE5F7E0B1E0BBBF5B
:10397C00B791BB2311F00E94225C17B1412F0E941A
:10398C005D5D1DE00E94FE611AE00E94FE61DF9108
:10399C00CF91CF93DF9318E0912A0BE71EE41A9393
:1039AC000A93E5E6F7E0B1E0BBBFB791BB2311F09A
:1039BC000E94225C16B1412F0E945D5D1DE00E94A9
:1039CC00FE611AE00E94FE61DF91CF91CF93DF93ED
:1039DC0018E0912A0BE71EE41A930A93EFE6F7E03E
:1039EC00B1E0BBBFB791BB2311F00E94225C15B1B3
:1039FC00412F0E945D5D1DE00E94FE611AE00E9455
:103A0C00FE61DF91CF91CF93DF9318E0912A0BE702
:103A1C001EE41A930A93E9E7F7E0B1E0BBBFB79154
:103A2C00BB2311F00E94225C14B1412F0E945D5DFA
:103A3C001DE00E94FE611AE00E94FE61DF91CF91B1
:103A4C00CF93DF9318E0912A0BE71EE41A930A93A5
:103A5C00E3E8F7E0B1E0BBBFB791BB2311F00E94E4
:103A6C00225C13B1412F0E945D5D1DE00E94FE613E
:103A7C001AE00E94FE61DF91CF91CF93DF9318E0A3
:103A8C00912A0BE71EE41A930A93EDE8F7E0B1E0F4
:103A9C00BBBFB791BB2311F00E94225C12B1412F26
:103AAC000E945D5D1DE00E94FE611AE00E94FE61B5
:103ABC00DF91CF91CF93DF9318E0912A0BE71EE4AF
:103ACC001A930A93E7E9F7E0B1E0BBBFB791BB23C8
:103ADC0011F00E94225C11B1412F0E945D5D1DE02E
:103AEC000E94FE611AE00E94FE61DF91CF91CF939C
:103AFC00DF9318E0912A0BE71EE41A930A93E1EA8C
:103B0C00F7E0B1E0BBBFB791BB2311F00E94225C80
:103B1C0010B1412F0E945D5D1DE00E94FE611AE014
:103B2C000E94FE61DF91CF91089510913E06109393
:103B3C00AD0210912006112311F40C94B41DCF93F7
:103B4C00DF9310913E061A930E94B90EDF91CF912C
:103B5C00F89410E01093200697FC789410911E06B0
:103B6C00112311F40C942D1E0E946F4E112311F48D
:103B7C000C94061E0E944D4EF8941093160697FC5A
:103B8C00789410911606113110E009F41FEF1123EF
:103B9C0011F40C94F21DCF93DF9318E0912A0BE7EC
:103BAC001EE41A930A93EBEAF7E0B1E0BBBFB791BE
:103BBC00BB2311F00E94225C1DE00E94FE611AE002
:103BCC000E94FE61DF91CF91F89410E010931E06D5
:103BDC0097FC78940C94061E10913F061093AD023E
:103BEC00CF93DF9318E0912A0BE71EE41A930A9304
:103BFC00109116060E94FE6197FC7894DF91CF918C
:103C0C0010913F061093AD020E946F4E112311F4D8
:103C1C000C942B1E0E944D4EF8941093160697FC94
:103C2C00789410913E061093AD02CF93DF9318E079
:103C3C00912A0BE71EE41A930A93109116060E9420
:103C4C00FE6197FC7894DF91CF910C94902ACF93DE
:103C5C00DF9318E0912A0BE71EE41A930A931DE0F8
:103C6C000E94FE611AE00E94FE61DF91CF91CF931A
:103C7C00DF9318E0912A0BE71EE41A930A93E1EC08
:103C8C00F7E0B1E0BBBFB791BB2311F00E94225CFF
:103C9C00DF91CF9120E030E0E9E6F1E010811123D3
:103CAC0029F40E94C75AE9E6F1E01081112309F0CA
:103CBC001FEFE8E2F6E0319610E2F894108397FCDF
:103CCC007894CF93DF93E8E2F6E08F011A930A938E
:103CDC001FE01A930E94700ADF91CF91E8E2F6E0A0
:103CEC0031961081113110E009F41FEF112311F4FA
:103CFC000C94BB1ECF93DF9318E0912A0BE71EE4C4
:103D0C001A930A931DE00E94FE611AE00E94FE6164
:103D1C00DF91CF9110911E06103010E009F41FEFC7
:103D2C00112311F40C94B91ECF93DF9318E0912A50
:103D3C000BE71EE41A930A93E4ECF7E0B1E0BBBF87
:103D4C00B791BB2311F00E94225C1DE00E94FE6122
:103D5C001AE00E94FE61DF91CF91F8941FEF10934F
:103D6C001E0697FC78940C94902ACF93DF9360975F
:103D7C00FE01EF93FF933196FA93EA931FE01A93A7
:103D8C0017EF91221FEB9122E8E2F6E0F8940E94E3
:103D9C002A5C97FC78941FE01F9318810F91011BEC
:103DAC00102FFF91EF91108323960E949308DF91BF
:103DBC00CF91F8941093170697FC789410911706EE
:103DCC00113011F00C940C1F0E944A0D10E0712F51
:103DDC00ABE9B4E042EA54E002E00E940764F894D4
:103DEC0011271093ED081093EC0810E01093E908DC
:103DFC0097FC7894F2011091EE080581101711F4DC
:103E0C000E94B65A97FC78940C94902A123011F0B8
:103E1C000C94321F0E944A0D10E0712FABE9B4E0F4
:103E2C0042EA54E002E00E940764F89411271093D0
:103E3C00ED081093EC0810E01093E90897FC7894C7
:103E4C00F2011091EE080581101711F40E94B65A78
:103E5C0097FC78940C94902A133011F00C94C21F98
:103E6C00CF93DF9318E0912A0BE71EE41A930A9381
:103E7C001DE00E94FE611AE00E94FE61DF91CF916D
:103E8C00CF93DF93E8E2F6E08F011A930A930E9436
:103E9C00DF06DF91CF91F89410931F0697FC78946E
:103EAC0010911F06112311F40C94731FCF93DF9301
:103EBC0018E0912A0BE71EE41A930A93E8E2F6E065
:103ECC00F8940E942A5C97FC78941DE00E94FE6195
:103EDC001AE00E94FE61DF91CF9110911F061F9393
:103EEC00CF93DF93E8E2F6E08F011A930A930E94D6
:103EFC000507DF91CF910F91102BF89410931F06AB
:103F0C0097FC789410911F06112311F40C94A71FA1
:103F1C00CF93DF9318E0912A0BE71EE41A930A93D0
:103F2C00E8E2F6E0F8940E942A5C97FC78941DE095
:103F3C000E94FE611AE00E94FE61DF91CF910C9409
:103F4C00C01FCF93DF9318E0912A0BE71EE41A935E
:103F5C000A93E9EDF7E0B1E0BBBFB791BB2311F0D9
:103F6C000E94225C1DE00E94FE611AE00E94FE612C
:103F7C00DF91CF910C94902A143011F00C94F7200F
:103F8C00CF93DF9318E0912A0BE71EE41A930A9360
:103F9C001DE00E94FE611AE00E94FE61DF91CF914C
:103FAC00CF93DF9318E0912A0BE71EE41A930A9340
:103FBC00EAEFF7E0B1E0BBBFB791BB2311F00E9471
:103FCC00225CDF91CF91CF93DF93CF93DF930E944D
:103FDC00E908DF91CF911A930E941F02DF91CF91D4
:103FEC00112311F40C94DC20CF93DF9318E0912A69
:103FFC000BE71EE41A930A93E0E0F8E0B1E0BBBFD4
:10400C00B791BB2311F00E94225CDF91CF91CF932B
:10401C00DF93CF93DF930E94E908DF91CF911A933E
:10402C000E945C02DF91CF91CF93DF9318E0912A2D
:10403C000BE71EE41A930A93E5E0F8E0B1E0BBBF8E
:10404C00B791BB2311F00E94225CDF91CF91CF93EB
:10405C00DF93CF93DF930E94E908DF91CF911A93FE
:10406C000E949902DF91CF91CF93DF9318E0912AB0
:10407C000BE71EE41A930A93EAE0F8E0B1E0BBBF49
:10408C00B791BB2311F00E94225CDF91CF91CF93AB
:10409C00DF93CF93DF930E94E908DF91CF911A93BE
:1040AC000E94EC01DF91CF91CF93DF9318E0912A1E
:1040BC000BE71EE41A930A931DE00E94FE611AE0BE
:1040CC000E94FE61DF91CF91CF93DF9318E0912A8C
:1040DC000BE71EE41A930A93EFE0F8E0B1E0BBBFE4
:1040EC00B791BB2311F00E94225CDF91CF91CF934B
:1040FC00DF93CF93DF930E94E908DF91CF911A935E
:10410C000E943501DF91CF91CF93DF9318E0912A74
:10411C000BE71EE41A930A93E0E0F8E0B1E0BBBFB2
:10412C00B791BB2311F00E94225CDF91CF91CF930A
:10413C00DF93CF93DF930E94E908DF91CF911A931D
:10414C000E947201DF91CF91CF93DF9318E0912AF7
:10415C000BE71EE41A930A93E3E1F8E0B1E0BBBF6E
:10416C00B791BB2311F00E94225CDF91CF91CF93CA
:10417C00DF93CF93DF930E94E908DF91CF911A93DD
:10418C000E94AF01DF91CF91CF93DF9318E0912A7A
:10419C000BE71EE41A930A931DE00E94FE611AE0DD
:1041AC000E94FE61DF91CF910C94F520CF93DF93A9
:1041BC0018E0912A0BE71EE41A930A93E8E1F8E061
:1041CC00B1E0BBBFB791BB2311F00E94225C1DE094
:1041DC000E94FE611AE00E94FE61DF91CF910C9467
:1041EC00902A153011F00C948621CF93DF9318E0B0
:1041FC00912A0BE71EE41A930A931DE00E94FE61BC
:10420C001AE00E94FE61DF91CF91CF93DF9318E00B
:10421C00912A0BE71EE41A930A93E9E3F8E0B1E064
:10422C00BBBFB791BB2311F00E94225CDF91CF91F1
:10423C00CF93DF930E949C09DF91CF91012F11271F
:10424C00A0E0B1E0E89495F80E946A620F931F9386
:10425C00CF93DF930E949C09DF91CF91012F1127FF
:10426C003F912F91020F131FF89400931C0610938B
:10427C001D0697FC7894CF93DF9318E0912A0BE7F7
:10428C001EE41A930A931DE00E94FE611AE00E943C
:10429C00FE61DF91CF91CF93DF9318E0912A0BE76A
:1042AC001EE41A930A93EBE4F8E0B1E0BBBFB791BC
:1042BC00BB2311F00E94225CDF91CF91F89410E5A2
:1042CC0097FC78941F93F89400911C0610911D068E
:1042DC0097FC78940F931F93689490F8CF93DF9387
:1042EC000E949C09DF91CF91E6E1F0E0612FA1E003
:1042FC00B0E03F912F914F910E94224E0C94902A46
:10430C00163011F00C945122CF93DF9318E0912AC0
:10431C000BE71EE41A930A931DE00E94FE611AE05B
:10432C000E94FE61DF91CF91CF93DF9318E0912A29
:10433C000BE71EE41A930A93E9E3F8E0B1E0BBBF84
:10434C00B791BB2311F00E94225CDF91CF91CF93E8
:10435C00DF930E949C09DF91CF91012F1127A0E0E0
:10436C00B1E0E89495F80E946A620F931F93CF9383
:10437C00DF930E949C09DF91CF91012F11273F9170
:10438C002F91020F131FF89400931C0610931D0617
:10439C0097FC7894CF93DF9318E0912A0BE71EE4F7
:1043AC001A930A931DE00E94FE611AE00E94FE61BE
:1043BC00DF91CF91CF93DF9318E0912A0BE71EE4A6
:1043CC001A930A93EEE5F8E0B1E0BBBFB791BB23BB
:1043DC0011F00E94225C1DE00E94FE611AE00E9416
:1043EC00FE61DF91CF910E944D4EF894109316060A
:1043FC0097FC7894CF93DF9318E0912A0BE71EE497
:10440C001A930A93109116060E94FE6197FC7894F9
:10441C00DF91CF91F89410E597FC78941F93F89462
:10442C0000911C0610911D0697FC78940F931F9316
:10443C00689490F8E6E1F6E0A1E0B0E03F912F91AE
:10444C004F910E94224EF894A0911C06B0911D062B
:10445C001196A0931C06B0931D0697FC78941091AE
:10446C0016061D3010E009F41FEF112311F40C9403
:10447C00F921CF93DF9318E0912A0BE71EE41A93EE
:10448C000A931DE00E94FE611AE00E94FE61DF911A
:10449C00CF910C94902A173011F00C94BC22CF932E
:1044AC00DF9318E0912A0BE71EE41A930A931DE0A0
:1044BC000E94FE611AE00E94FE61DF91CF91CF93C2
:1044CC00DF9318E0912A0BE71EE41A930A93E9E3B1
:1044DC00F8E0B1E0BBBFB791BB2311F00E94225CA6
:1044EC00DF91CF91CF93DF930E949C09DF91CF9105
:1044FC00012F1127A0E0B1E0E89495F80E946A62C0
:10450C000F931F93CF93DF930E949C09DF91CF9160
:10451C00012F11273F912F91020F131FF894009335
:10452C001C0610931D0697FC7894CF93DF9318E02C
:10453C00912A0BE71EE41A930A931DE00E94FE6178
:10454C001AE00E94FE61DF91CF91CF93DF93F89434
:10455C0000911C0610911D0697FC78941A930A93EF
:10456C000E94DD0ADF91CF910C94902A183011F043
:10457C000C942625CF93DF9318E0912A0BE71EE4C9
:10458C001A930A931DE00E94FE611AE00E94FE61DC
:10459C00DF91CF91CF93DF9318E0912A0BE71EE4C4
:1045AC001A930A93E5E7F8E0B1E0BBBFB791BB23E0
:1045BC0011F00E94225CDF91CF91CF93DF93E8E35F
:1045CC00F6E08F011A930A9311E01A930E94700A75
:1045DC00DF91CF91CF93DF9318E0912A0BE71EE484
:1045EC001A930A931DE00E94FE611AE00E94FE617C
:1045FC00DF91CF91E8E3F6E03196EF93FF93E8E398
:10460C00F6E031961081113618F01B3708F4105271
:10461C00F894FF91EF91119397FC7894E8E3F6E00E
:10462C0031961081163431F020F4113410F04427F7
:10463C0001C041E010E009F41FEF112311F40C94B8
:10464C000B25CF93DF9318E0912A0BE71EE41A9306
:10465C000A931DE00E94FE611AE00E94FE61DF9148
:10466C00CF91CF93DF9318E0912A0BE71EE41A93B6
:10467C000A93E3E8F8E0B1E0BBBFB791BB2311F0BC
:10468C000E94225CE8E3F6E0F8940E942A5C97FC16
:10469C007894E8E8F8E0B1E0BBBFB791BB2311F028
:1046AC000E94225C1DE00E94FE611AE00E94FE61E5
:1046BC00DF91CF91CF93DF9318E0912A0BE71EE4A3
:1046CC001A930A93E4E9F8E0B1E0BBBFB791BB23BE
:1046DC0011F00E94225C1DE00E94FE611AE00E9413
:1046EC00FE61DF91CF91CF93DF9318E0912A0BE716
:1046FC001EE41A930A93E0ECF8E0B1E0BBBFB7916B
:10470C00BB2311F00E94225CE8E3F6E0F8940E94CF
:10471C002A5C97FC7894E4ECF8E0B1E0BBBFB7916D
:10472C00BB2311F00E94225CDF91CF91E8E3F6E00D
:10473C0031961081113411F00C94AE23CF93DF938A
:10474C001AB31A930E941B0CDF91CF910C94F52392
:10475C00123411F00C94BC23CF93DF9317B31A933C
:10476C000E941B0CDF91CF910C94F523133411F0A4
:10477C000C94CA23CF93DF9314B31A930E941B0C8F
:10478C00DF91CF910C94F523143411F00C94D823B1
:10479C00CF93DF9311B31A930E941B0CDF91CF912F
:1047AC000C94F523153411F00C94E623CF93DF937E
:1047BC0012B11A930E941B0CDF91CF910C94F5232C
:1047CC00163411F00C94F523CF93DF931091610004
:1047DC001A930E941B0CDF91CF910C94F523CF936D
:1047EC00DF9318E0912A0BE71EE41A930A931DE05D
:1047FC000E94FE611AE00E94FE61DF91CF91CF937F
:10480C00DF9318E0912A0BE71EE41A930A93EBEC62
:10481C00F8E0B1E0BBBFB791BB2311F00E94225C62
:10482C00DF91CF91E8E3F6E031961081113411F06D
:10483C000C942C24CF93DF931AB31A931BB31A93B3
:10484C000E94CB0CDF91CF910C947E24123411F08A
:10485C000C943C24CF93DF9317B31A9318B31A9389
:10486C000E94CB0CDF91CF910C947E24133411F069
:10487C000C944C24CF93DF9314B31A9315B31A935F
:10488C000E94CB0CDF91CF910C947E24143411F048
:10489C000C945C24CF93DF9311B31A9312B31A9335
:1048AC000E94CB0CDF91CF910C947E24153411F027
:1048BC000C946C24CF93DF9312B11A9313B11A9307
:1048CC000E94CB0CDF91CF910C947E24163411F006
:1048DC000C947E24CF93DF93109161001A93109166
:1048EC0062001A930E94CB0CDF91CF910C947E2422
:1048FC00CF93DF9318E0912A0BE71EE41A930A93E7
:10490C001DE00E94FE611AE00E94FE61DF91CF91D2
:10491C00CF93DF9318E0912A0BE71EE41A930A93C6
:10492C00E6EDF8E0B1E0BBBFB791BB2311F00E94FC
:10493C00225CDF91CF91E8E3F6E0319610811134DF
:10494C0011F00C94B324CF93DF9319B31A930E94F4
:10495C00730CDF91CF910C94F924123411F00C9458
:10496C00C124CF93DF9316B31A930E94730CDF917B
:10497C00CF910C94F924133411F00C94CF24CF93D1
:10498C00DF9313B31A930E94730CDF91CF910C94A5
:10499C00F924143411F00C94DD24CF93DF9310B36D
:1049AC001A930E94730CDF91CF910C94F924153457
:1049BC0011F00C94EB24CF93DF9311B11A930E9456
:1049CC00730CDF91CF910C94F924163411F00C94E4
:1049DC00F924CF93DF9310B11A930E94730CDF91DB
:1049EC00CF910C94F924CF93DF9318E0912A0BE725
:1049FC001EE41A930A931DE00E94FE611AE00E94C5
:104A0C00FE61DF91CF910C942425CF93DF9318E0B6
:104A1C00912A0BE71EE41A930A93E1EEF8E0B1E059
:104A2C00BBBFB791BB2311F00E94225C1DE00E941A
:104A3C00FE611AE00E94FE61DF91CF910C94902AE6
:104A4C00193011F00C944E28CF93DF9318E0912A73
:104A5C000BE71EE41A930A931DE00E94FE611AE014
:104A6C000E94FE61DF91CF91CF93DF9318E0912AE2
:104A7C000BE71EE41A930A93E3EFF8E0B1E0BBBF37
:104A8C00B791BB2311F00E94225CDF91CF91CF93A1
:104A9C00DF93E8E3F6E08F011A930A9312E01A937E
:104AAC000E94700ADF91CF91CF93DF9318E0912A87
:104ABC000BE71EE41A930A931DE00E94FE611AE0B4
:104ACC000E94FE61DF91CF91E8E3F6E03196EF931F
:104ADC00FF93E8E3F6E031961081113618F01B379E
:104AEC0008F41052F894FF91EF91119397FC78947D
:104AFC00E8E3F6E031961081163431F020F41134ED
:104B0C0010F0442701C041E010E009F41FEF11231D
:104B1C0011F40C943328F8941FEF10931A0697FC99
:104B2C007894E8E3F6E031961081113411F00C948E
:104B3C00A72510E00AE300936105109362050C941D
:104B4C00EF25123411F00C94B32510E007E3009319
:104B5C006105109362050C94EF25133411F00C943D
:104B6C00BF2510E004E300936105109362050C94DB
:104B7C00EF25143411F00C94D12510E001E30093CF
:104B8C00610510936205F89410EF10931A0697FCC8
:104B9C0078940C94EF25153411F00C94E32510E067
:104BAC0002E20093610510936205F8941CEF1093D8
:104BBC001A0697FC78940C94EF25163411F00C948B
:104BCC00EF2510E001E600936105109362050C944B
:104BDC00EF25CF93DF9318E0912A0BE71EE41A938D
:104BEC000A93E2E0F9E0B1E0BBBFB791BB2311F04F
:104BFC000E94225CDF91CF91CF93DF930E94E90852
:104C0C00DF91CF91F8941093190697FC7894CF9379
:104C1C00DF9318E0912A0BE71EE41A930A931DE028
:104C2C000E94FE611AE00E94FE61DF91CF9110910B
:104C3C001906173031F020F4103010F0442701C061
:104C4C0041E010E009F41FEF112311F40C94182823
:104C5C0010911A061F9310911906212F11E00E9432
:104C6C0037620F911023F89410931B0697FC7894DD
:104C7C0010911B06103010E011F008F01FEF1123FB
:104C8C0011F40C94ED27CF93DF9318E0912A0BE7E6
:104C9C001EE41A930A93EEE0F9E0B1E0BBBFB791C2
:104CAC00BB2311F00E94225CDF91CF91CF93DF9355
:104CBC00EBE3F6E08F011A930A9312E01A930E9429
:104CCC00700ADF91CF91CF93DF9318E0912A0BE715
:104CDC001EE41A930A931DE00E94FE611AE00E94E2
:104CEC00FE61DF91CF91EBE3F6E03196EF93FF930A
:104CFC00EBE3F6E031961081113618F01B3708F40F
:104D0C001052F894FF91EF91119397FC7894EBE388
:104D1C00F6E031961081193410E009F41FEF1F935F
:104D2C00EBE3F6E0319610811F3410E009F41FEF2D
:104D3C000F91102B112311F40C94D227EBE3F6E016
:104D4C0031961081193410E009F41FEF112311F47E
:104D5C000C94BD27E0916105F0916205EF93FF93F0
:104D6C00E0916105F091620510811F9310911B0673
:104D7C0010950F911023FF91EF911193CF93DF9327
:104D8C0018E0912A0BE71EE41A930A93E4E1F9E088
:104D9C00B1E0BBBFB791BB2311F00E94225CDF9145
:104DAC00CF91CF93DF93EBE3F6E08F011A930A9345
:104DBC0012E01A930E94700ADF91CF91CF93DF9388
:104DCC0018E0912A0BE71EE41A930A931DE00E9447
:104DDC00FE611AE00E94FE61DF91CF91EBE3F6E0F9
:104DEC003196EF93FF93EBE3F6E031961081113699
:104DFC0018F01B3708F41052F894FF91EF911193AF
:104E0C0097FC7894EBE3F6E0319610811E3410E0B9
:104E1C0009F41FEF1F93EBE3F6E03196108119357F
:104E2C0010E009F41FEF0F91102B112311F40C94C7
:104E3C00A227E8E3F6E031961081113411F00C94BE
:104E4C002F2710E00BE300936105109362050C947F
:104E5C006B27123411F00C943B2710E008E30093FD
:104E6C006105109362050C946B27133411F00C94AC
:104E7C00472710E005E300936105109362050C943D
:104E8C006B27143411F00C94532710E002E30093B9
:104E9C006105109362050C946B27153411F00C947A
:104EAC005F2710E003E200936105109362050C94F8
:104EBC006B27163411F00C946B2710E002E600936C
:104ECC006105109362050C946B27EBE3F6E03196C9
:104EDC0010811E3410E009F41FEF112311F40C940F
:104EEC008D27E0916105F0916205EF93FF93E091BE
:104EFC006105F091620510811F9310911B061095AE
:104F0C000F911023FF91EF9111930C94A027E09136
:104F1C006105F0916205EF93FF93E0916105F091CB
:104F2C00620510811F9310911B060F91102BFF919E
:104F3C00EF9111930C94BB27CF93DF9318E0912A38
:104F4C000BE71EE41A930A93EBE2F9E0B1E0BBBF66
:104F5C00B791BB2311F00E94225C1DE00E94FE6100
:104F6C001AE00E94FE61DF91CF910C94D027E09162
:104F7C006105F0916205EF93FF93E0916105F0916B
:104F8C00620510811F9310911B060F91102BFF913E
:104F9C00EF9111930C94EB27CF93DF9318E0912AA8
:104FAC000BE71EE41A930A93EFE3F9E0B1E0BBBF01
:104FBC00B791BB2311F00E94225C1DE00E94FE61A0
:104FCC001AE00E94FE61DF91CF910C941628CF93CA
:104FDC00DF9318E0912A0BE71EE41A930A931DE065
:104FEC000E94FE611AE00E94FE61DF91CF91CF9387
:104FFC00DF9318E0912A0BE71EE41A930A93E0E57D
:10500C00F9E0B1E0BBBFB791BB2311F00E94225C69
:10501C001DE00E94FE611AE00E94FE61DF91CF91BB
:10502C000C943128CF93DF9318E0912A0BE71EE400
:10503C001A930A93E0E7F9E0B1E0BBBFB791BB2349
:10504C0011F00E94225C1DE00E94FE611AE00E9499
:10505C00FE61DF91CF910C944C28CF93DF9318E035
:10506C00912A0BE71EE41A930A93E1EEF8E0B1E003
:10507C00BBBFB791BB2311F00E94225C1DE00E94C4
:10508C00FE611AE00E94FE61DF91CF910C94902A90
:10509C001A3011F00C94312ACF93DF9318E0912A37
:1050AC000BE71EE41A930A931DE00E94FE611AE0BE
:1050BC000E94FE61DF91CF91CF93DF9318E0912A8C
:1050CC000BE71EE41A930A93E3EFF8E0B1E0BBBFE1
:1050DC00B791BB2311F00E94225CDF91CF91CF934B
:1050EC00DF93E8E3F6E08F011A930A9312E01A9328
:1050FC000E94700ADF91CF91CF93DF9318E0912A31
:10510C000BE71EE41A930A931DE00E94FE611AE05D
:10511C000E94FE61DF91CF91E8E3F6E03196EF93C8
:10512C00FF93E8E3F6E031961081113618F01B3747
:10513C0008F41052F894FF91EF91119397FC789426
:10514C00E8E3F6E031961081163431F020F4113496
:10515C0010F0442701C041E010E009F41FEF1123C7
:10516C0011F40C94062AF8941FEF10931A0697FC6E
:10517C007894E8E3F6E031961081113411F00C9438
:10518C00CF2810E00BE300936105109362050C949B
:10519C001729123411F00C94DB2810E008E300936B
:1051AC006105109362050C941729133411F00C94BB
:1051BC00E72810E005E300936105109362050C9459
:1051CC001729143411F00C94F92810E002E3009321
:1051DC00610510936205F89410EF10931A0697FC72
:1051EC0078940C941729153411F00C940B2910E0B9
:1051FC0003E20093610510936205F8941CEF109381
:10520C001A0697FC78940C941729163411F00C9408
:10521C00172910E002E600936105109362050C94C7
:10522C001729CF93DF9318E0912A0BE71EE41A930A
:10523C000A93E1E8F9E0B1E0BBBFB791BB2311F0F1
:10524C000E94225CDF91CF91CF93DF930E94E908FB
:10525C00DF91CF91F8941093190697FC7894CF9323
:10526C00DF9318E0912A0BE71EE41A930A931DE0D2
:10527C000E94FE611AE00E94FE61DF91CF911091B5
:10528C001906173031F020F4103010F0442701C00B
:10529C0041E010E009F41FEF112311F40C94EB29F9
:1052AC0010911A061F9310911906212F11E00E94DC
:1052BC0037620F911023F89410931B0697FC789487
:1052CC0010911B06103010E011F008F01FEF1123A5
:1052DC0011F40C94C029CF93DF9318E0912A0BE7BB
:1052EC001EE41A930A93EEE8F9E0B1E0BBBFB79164
:1052FC00BB2311F00E94225CDF91CF91CF93DF93FF
:10530C000E94E908DF91CF91112309F01FEF1F3F95
:10531C0010E009F41FEF112311F40C94AA29E09169
:10532C006105F0916205EF93FF93E0916105F091B7
:10533C00620510811F9310911B060F91102BFF918A
:10534C00EF9111930C94BE29E0916105F0916205E7
:10535C00EF93FF93E0916105F091620510811F932B
:10536C0010911B0610950F911023FF91EF91119343
:10537C000C94E929CF93DF9318E0912A0BE71EE4F4
:10538C001A930A931DE00E94FE611AE00E94FE61CE
:10539C00DF91CF91CF93DF9318E0912A0BE71EE4B6
:1053AC001A930A93E0E5F9E0B1E0BBBFB791BB23D8
:1053BC0011F00E94225C1DE00E94FE611AE00E9426
:1053CC00FE61DF91CF910C94042ACF93DF9318E008
:1053DC00912A0BE71EE41A930A93E5E9F9E0B1E090
:1053EC00BBBFB791BB2311F00E94225C1DE00E9451
:1053FC00FE611AE00E94FE61DF91CF910C941F2A8E
:10540C00CF93DF9318E0912A0BE71EE41A930A93CB
:10541C00E1EEF8E0B1E0BBBFB791BB2311F00E9405
:10542C00225C1DE00E94FE611AE00E94FE61DF9189
:10543C00CF91CF93DF9318E0912A0BE71EE41A93D8
:10544C000A931DE00E94FE611AE00E94FE61DF914A
:10545C00CF910C94902A1B3011F00C943D2ACF93D1
:10546C00DF930E94920FDF91CF910C94902ACF93EF
:10547C00DF936097FE01EF93FF933196FA93EA93D3
:10548C001FE01A9317EF91221FEB9122E8E2F6E04E
:10549C00F8940E942A5C97FC78941FE01F93188163
:1054AC000F91011B102FFF91EF91108323960E94F7
:1054BC003A08DF91CF91F8941093170697FC7894E3
:1054CC0010911706103010E011F008F01FEF1123A7
:1054DC0011F40C94902A10911706712FABE9B4E0DB
:1054EC0042EA54E002E00E940764F89411271093FA
:1054FC00ED081093EC0810E01093E90897FC7894F1
:10550C00F2011091EE080581101711F40E94B65AA1
:10551C0097FC78940C949B1D1881103010E009F4C2
:10552C001FEF112311F40C94A92AF89410E0109396
:10553C003E0697FC7894F89411E010933F0697FC84
:10554C0078940C94B52AF89411E010933E0697FCCD
:10555C007894F89410E010933F0697FC7894CF93CE
:10556C00DF9318811A930E94B90EDF91CF910895A1
:10557C00F89410E010931E0697FC7894F8941FEFA3
:10558C001093200697FC7894F89410E010933E0644
:10559C0097FC7894F89411E010933F0697FC78945C
:1055AC0010E000E000935D0510935E0510E0109391
:1055BC005F0510E0109360050895219710E0E981D4
:1055CC00FA8110831D81173031F020F4103010F067
:1055DC00442701C041E010E009F41FEF112311F43E
:1055EC000C94182B1D8110651D831D811F930B813D
:1055FC001C819801689490F84F91A0E0B0E00E9453
:10560C00224E188318811F931D811F93E981FA8103
:10561C00A1E0B0E04F910E94104E0F91102B188317
:10562C000C941A2B10E018831881089521971C8173
:10563C00173031F020F4103010F0442701C041E055
:10564C0010E009F41FEF112311F40C94442B1C816E
:10565C0010651C831C811F930A811B810F931F9360
:10566C00689490F8FE013196A1E0B0E03F912F9143
:10567C004F910E94224E18830C94462B10E01883F5
:10568C001881089518811F930F91100F1150012F3D
:10569C001127009344061093450608952397009113
:1056AC00440610914506103009F4003010E011F05A
:1056BC0008F01FEF112311F40C94212C1A851030D3
:1056CC0011F00C946D2B1FEF1A830C941F2C1130BE
:1056DC0011F00C94752B1FEF1A830C941F2C1230A5
:1056EC0011F00C94A12B0F8118850F931F9300912F
:1056FC0044061091450698011F910F91131709F458
:10570C0002171FEF08F01127112311F40C949D2B95
:10571C000F811885102F1093420610914206169592
:10572C00105B109343061FEF1A830C949F2B10E011
:10573C001A830C941F2C133011F00C94C52B0F8171
:10574C001885A12F102F0A2F169507950093400648
:10575C0010934106A0E4B6E0AF93BF931EE01F93F5
:10576C0010914206A12F1127A0FD1FEF0F91BF91A1
:10577C00AF910E94C5631FEF1A830C941F2C143039
:10578C0011F00C94F32B0F81188519830883109159
:10579C0043061F93009140061091410698016894AE
:1057AC0090F84F91A0E0B0E00E94224E1A831A812B
:1057BC001F93109143061F93E881F981EF93FF9398
:1057CC0010E000E8D801FF91EF914F910E94104E2C
:1057DC000F91102B1A830C941F2C153011F00C9474
:1057EC00172C0F81188519830883109143061F937A
:1057FC0000914006109141060F931F93689490F806
:10580C00E881F981EF93FF9310E000E8D801FF9154
:10581C00EF913F912F914F910E94224E1A830C943D
:10582C001F2C163011F00C941F2C1FEF1A830C94A4
:10583C001F2C0C94232C10E01A831A81089510E06D
:10584C0000E0009340061093410610E010934206CE
:10585C0010E01093430610E000E000934406109310
:10586C0045060895229710E019831B81173031F0FB
:10587C0020F4103010F0442701C041E010E009F48E
:10588C001FEF112311F40C945A2C1B81105E1883FA
:10589C0018811F931A81312FE89490F84F91A0E052
:1058AC00B0E00E94224E198319810895229710E0CE
:1058BC00EA81FB81108310E019831C81173031F0D1
:1058CC0020F4103010F0442701C041E010E009F43E
:1058DC001FEF112311F40C94902C1C81105E188373
:1058EC0018811F931FEF312FE89490F84F91A0E08F
:1058FC00B0E00E94224E198319811F9318811F93C7
:10590C00EA81FB81A1E0B0E04F910E94104E0F9113
:10591C00102B1983198108950895229710E018838C
:10592C00FE013196FA93EA9310E0108317E01A9374
:10593C001081088101171FEF08F01127112311F0B6
:10594C000C94C32C1B811F931D811F931C810E94DF
:10595C00416211701F931C8107E0011B102F0E94E4
:10596C0031620F91102B1B83E981FA811081139501
:10597C001083112311F00C949F2C239618810895F9
:10598C002197FE013196EF93FF933196FA93EA93A8
:10599C0010E11A9317EF91221FEB9122FE0134961E
:1059AC00EF93FF9310E100E20A93FF91EF91EF93D5
:1059BC00FF930981101708F0102F0191FF91EF91BF
:1059CC00101B08F411271F9319911F93102F01E03E
:1059DC000E940E5C1F91EF91EE2321F00E94FE615C
:1059EC00EA95E1F710E11F9318810F91011B102F1D
:1059FC00FF91EF9110832396CF93DF9310E01A93CE
:105A0C00E4E2F0E1EF93FF931B89012F1127FF9143
:105A1C00EF91E00FF11F16911A930E94314DDF9117
:105A2C00CF91FE01FA93EA9311E0108318E01A93D8
:105A3C001081088101171FEF08F01127112311F0B5
:105A4C000C94492DCF93DF9318E0912A0FE71CE4B7
:105A5C001A930A93FE013696EF93FF931D81FF91E3
:105A6C00EF91012F1127E00FF11F10810E94FE61B1
:105A7C00DF91CF91E981FA81108113951083112365
:105A8C0011F00C941F2D2396CF93DF9310E41A93EF
:105A9C00E4E2F0E1EF93FF931B89012F1127FF91B3
:105AAC00EF91E00FF11F16911A930E94314DDF9187
:105ABC00CF91FE01FA93EA9319E0108310E11A9347
:105ACC001081088101171FEF08F01127112311F025
:105ADC000C94912DCF93DF9318E0912A0FE71CE4DF
:105AEC001A930A93FE013696EF93FF931D81FF9153
:105AFC00EF91012F1127E00FF11F10810E94FE6121
:105B0C00DF91CF91E981FA811081139510831123D4
:105B1C0011F00C94672D2396089510E01F9310E05C
:105B2C001F930E94214D0E94474D10E003E00E94FC
:105B3C00295B0E94674D08952297FE013196FA93D6
:105B4C00EA9310E0108317E01A9310810881011773
:105B5C001FEF08F01127112311F00C94E72D1C8175
:105B6C00212F11E00E9437621B831B811F931E8122
:105B7C000F911023112309F01FEF1F3F10E009F4C0
:105B8C001FEF112311F40C94DE2DEF81F885EF93A8
:105B9C00FF931C811F931B811F931D810F91102359
:105BAC00112309F01FEF0F91BF91AF910E94B363C6
:105BBC00E981FA81108113951083112311F00C9453
:105BCC00AC2D23960895EC97CF93DF9310E01A93A6
:105BDC006197FE01EF93FF933196FA93EA9310E1EC
:105BEC001A9317EF91221FEB9122E6EAF9E0B1E04C
:105BFC00BBBFB791BB2311F00E94225C10E11F9335
:105C0C0018810F91011B102FFF91EF911083239698
:105C1C000E94C62CDF91CF91CF93DF9318E0912A8D
:105C2C000BE71EE41A930A931DE00E94FE611AE032
:105C3C000E94FE61DF91CF91CF93DF9318E0912A00
:105C4C000BE71EE41A930A93E7EBF9E0B1E0BBBF54
:105C5C00B791BB2311F00E94225C1DE00E94FE61F3
:105C6C001AE00E94FE61DF91CF9113E008EE0E94D2
:105C7C00295BCF93DF9318E0912A0BE71EE41A936C
:105C8C000A931DE00E94FE611AE00E94FE61DF9102
:105C9C00CF91CF93DF9310E01A936197FE01EF93AE
:105CAC00FF933196FA93EA9310E11A9317EF91222E
:105CBC001FEB9122EAEDF9E0B1E0BBBFB791BB233A
:105CCC0011F00E94225C10E11F9318810F91011BAF
:105CDC00102FFF91EF91108323960E94C62CDF9119
:105CEC00CF91CF93DF9318E0912A0BE71EE41A9320
:105CFC000A93EAEDF9E0B1E0BBBFB791BB2311F019
:105D0C000E94225CDF91CF9110E0E0E3F0E0EC0F19
:105D1C00FD1F1083FE01F796FA93EA9310E01083AF
:105D2C0013E61A931081088101171FEF08F0112751
:105D3C00112311F00C9469321FEF1ABB0E9485637A
:105D4C00102FEBE3F0E0EC0FFD1F1083CF93DF93EC
:105D5C00EBE3F0E0EC0FFD1F10811A930E94932CE3
:105D6C00DF91CF911BBBCF93DF9310E01A93FE0111
:105D7C00FF968F011A930A930E945C2CDF91CF91AE
:105D8C00EEE3F0E0EC0FFD1F10811F93EBE3F0E06E
:105D9C00EC0FFD1F10810F91011710E009F01FEFA0
:105DAC00112311F40C94E52EE3E3F0E0EC0FFD1F4E
:105DBC0010811068E3E3F0E0EC0FFD1F10831FEF80
:105DCC001BBB10E01ABB0E948563102FEBE3F0E0C5
:105DDC00EC0FFD1F1083CF93DF9310E01A93CF933A
:105DEC00DF93ECE3F0E0EC0FFD1F10811A930E949F
:105DFC00932CDF91CF911A930E94382CDF91CF9185
:105E0C0019B31F93EBE3F0E0EC0FFD1F10810F9122
:105E1C00011710E009F01FEF112311F40C94212F3E
:105E2C00E3E3F0E0EC0FFD1F10811068E3E3F0E01A
:105E3C00EC0FFD1F10831FEF17BB0E948563102F03
:105E4C00EBE3F0E0EC0FFD1F1083CF93DF93EBE35C
:105E5C00F0E0EC0FFD1F10811A930E94932CDF9140
:105E6C00CF9118BBCF93DF9311E01A93FE01FF96ED
:105E7C008F011A930A930E945C2CDF91CF91EEE371
:105E8C00F0E0EC0FFD1F10811F93EBE3F0E0EC0F43
:105E9C00FD1F10810F91011710E009F01FEF112366
:105EAC0011F40C94642FE3E3F0E0EC0FFD1F108170
:105EBC001064E3E3F0E0EC0FFD1F10831FEF18BB41
:105ECC0010E017BB0E948563102FEBE3F0E0EC0FA2
:105EDC00FD1F1083CF93DF9311E01A93CF93DF93C1
:105EEC00ECE3F0E0EC0FFD1F10811A930E94932C51
:105EFC00DF91CF911A930E94382CDF91CF9116B37A
:105F0C001F93EBE3F0E0EC0FFD1F10810F910117D5
:105F1C0010E009F01FEF112311F40C94A02FE3E310
:105F2C00F0E0EC0FFD1F10811064E3E3F0E0EC0FE8
:105F3C00FD1F1083CF93DF9310E001E31A930A93B4
:105F4C0010EF1A9310EF1A930E94A22DDF91CF91AC
:105F5C000E948563102F107FEBE3F0E0EC0FFD1F28
:105F6C001083CF93DF9310E002E31A930A9310EFA0
:105F7C001A93EEE3F0E0EC0FFD1F10811A930E94D0
:105F8C00A22DDF91CF91CF93DF9313E01A93FE01F3
:105F9C00FF968F011A930A930E945C2CDF91CF918C
:105FAC00CF93DF93EEE3F0E0EC0FFD1F10811A931B
:105FBC000E94932CDF91CF91107FEEE3F0E0EC0F79
:105FCC00FD1F1083EEE3F0E0EC0FFD1F10811F931B
:105FDC00EBE3F0E0EC0FFD1F10810F91011710E0C7
:105FEC0009F01FEF112311F40C940730E3E3F0E0F8
:105FFC00EC0FFD1F10811061E3E3F0E0EC0FFD1FCF
:10600C001083CF93DF9310E001E31A930A9310EF00
:10601C001A9310E01A930E94A22DDF91CF91CF9387
:10602C00DF9310E002E31A930A9310EF1A9310EF28
:10603C001A930E94A22DDF91CF910E948563102F9D
:10604C001F60EBE3F0E0EC0FFD1F1083CF93DF93A9
:10605C0013E01A93CF93DF93ECE3F0E0EC0FFD1F0A
:10606C0010811A930E94932CDF91CF911A930E9466
:10607C00382CDF91CF9110B3107F1F93EBE3F0E03E
:10608C00EC0FFD1F1081107F0F91011710E009F02C
:10609C001FEF112311F40C945E30E3E3F0E0EC0FEE
:1060AC00FD1F10811061E3E3F0E0EC0FFD1F108386
:1060BC00CF93DF9310E002E21A930A931CEF1A932A
:1060CC001CEF1A930E94A22DDF91CF910E94856341
:1060DC00102F1C7FEBE3F0E0EC0FFD1F1083CF9330
:1060EC00DF9310E003E21A930A931CEF1A93EEE38A
:1060FC00F0E0EC0FFD1F10811A930E94A22DDF918E
:10610C00CF91CF93DF9314E01A93FE01FF968F018A
:10611C001A930A930E945C2CDF91CF91CF93DF935B
:10612C00EEE3F0E0EC0FFD1F10811A930E94932C0C
:10613C00DF91CF911C7FEEE3F0E0EC0FFD1F10839D
:10614C00EEE3F0E0EC0FFD1F10811F93EBE3F0E0AA
:10615C00EC0FFD1F10810F91011710E009F01FEFDC
:10616C00112311F40C94C530E3E3F0E0EC0FFD1FA8
:10617C0010811860E3E3F0E0EC0FFD1F1083CF9368
:10618C00DF9310E002E21A930A931CEF1A9310E0CB
:10619C001A930E94A22DDF91CF91CF93DF9310E041
:1061AC0003E21A930A931CEF1A931CEF1A930E94A2
:1061BC00A22DDF91CF910E948563102F1360EBE32A
:1061CC00F0E0EC0FFD1F1083CF93DF9314E01A93D4
:1061DC00CF93DF93ECE3F0E0EC0FFD1F10811A93EB
:1061EC000E94932CDF91CF911A930E94382CDF914F
:1061FC00CF9111B11C7F1F93EBE3F0E0EC0FFD1F6F
:10620C0010811C7F0F91011710E009F01FEF112373
:10621C0011F40C941C31E3E3F0E0EC0FFD1F108142
:10622C001860E3E3F0E0EC0FFD1F10831FEF1093F9
:10623C0061000E948563102FEBE3F0E0EC0FFD1F73
:10624C001083CF93DF93EBE3F0E0EC0FFD1F108195
:10625C001A930E94932CDF91CF9110936200CF93ED
:10626C00DF9315E01A93FE01FF968F011A930A93A0
:10627C000E945C2CDF91CF91EEE3F0E0EC0FFD1F60
:10628C0010811F93EBE3F0E0EC0FFD1F10810F91D9
:10629C00011710E009F01FEF112311F40C94613178
:1062AC00E3E3F0E0EC0FFD1F10811460E3E3F0E09A
:1062BC00EC0FFD1F108310E0109361001FEF109383
:1062CC0062000E948563102FEBE3F0E0EC0FFD1FE2
:1062DC001083CF93DF9315E01A93CF93DF93ECE306
:1062EC00F0E0EC0FFD1F10811A930E94932CDF91AC
:1062FC00CF911A930E94382CDF91CF9110B11F933C
:10630C00EBE3F0E0EC0FFD1F10810F91011710E093
:10631C0009F01FEF112311F40C949F31E3E3F0E02B
:10632C00EC0FFD1F10811460E3E3F0E0EC0FFD1F98
:10633C0010830E948563102FEBE3F0E0EC0FFD1F40
:10634C001083CF93DF9315E01A93CF93DF93ECE395
:10635C00F0E0EC0FFD1F10811A930E94932CDF913B
:10636C00CF911A930E94382CDF91CF9110E00AE064
:10637C000E94295BFE01F996FA93EA9311E01083CF
:10638C0018E01A931081088101171FEF08F01127EC
:10639C00112311F00C945F32ECE3F0E0EC0FFD1FD5
:1063AC0010810E94DB630F7F1370EFE3F0E0EC0FC2
:1063BC00FD1F01931083EFE3F0E0EC0FFD1F019143
:1063CC001191689492F8A0E0B0E055270E94986370
:1063DC0055234AF4ACE3B0E055270E94986355234B
:1063EC0012F0112701C01FEF10E009F41FEF1F93EB
:1063FC00FE01FE96EF93FF93ECE3F0E0EC0FFD1F34
:10640C0010811150BF91AF910E94A663103010E023
:10641C0009F41FEF0F9110231F93EFE3F0E0EC0F43
:10642C00FD1F01911191689492F8A8EEB3E05527E5
:10643C000E94986355234AF4A0E0B4E055270E94CB
:10644C009863552312F0112701C01FEF10E009F4D7
:10645C001FEF1F93FE01FE96EF93FF93ECE3F0E02A
:10646C00EC0FFD1F10811150BF91AF910E94A663DC
:10647C001F3F10E009F41FEF0F9110230F91102B09
:10648C001095112311F40C945632E6E3F0E0EC0F66
:10649C00FD1F10811260E6E3F0E0EC0FFD1F10838E
:1064AC00E981FA81108113951083112311F00C945A
:1064BC00C9312396E981FA81108113951083112338
:1064CC0011F00C94992E2396CF93DF9318E0912A18
:1064DC000BE71EE41A930A931DE00E94FE611AE07A
:1064EC000E94FE61DF91CF91E0E3F0E0EC0FFD1F25
:1064FC001081103010E011F008F01FEF112311F48F
:10650C000C94CA33E0E3F0E0EC0FFD1F108110781F
:10651C00103010E011F008F01FEF112311F40C945F
:10652C00B032CF93DF9318E0912A0BE71EE41A9355
:10653C000A93E9EEF9E0B1E0BBBFB791BB2311F0D0
:10654C000E94225C1DE00E94FE611AE00E94FE6126
:10655C00DF91CF91E0E3F0E0EC0FFD1F10811074A0
:10656C00103010E011F008F01FEF112311F40C940F
:10657C00D832CF93DF9318E0912A0BE71EE41A93DD
:10658C000A93EAEFF9E0B1E0BBBFB791BB2311F07E
:10659C000E94225C1DE00E94FE611AE00E94FE61D6
:1065AC00DF91CF91E0E3F0E0EC0FFD1F1081107252
:1065BC00103010E011F008F01FEF112311F40C94BF
:1065CC000033CF93DF9318E0912A0BE71EE41A9364
:1065DC000A93EBE0FAE0B1E0BBBFB791BB2311F03B
:1065EC000E94225C1DE00E94FE611AE00E94FE6186
:1065FC00DF91CF91E0E3F0E0EC0FFD1F1081107103
:10660C00103010E011F008F01FEF112311F40C946E
:10661C002833CF93DF9318E0912A0BE71EE41A93EB
:10662C000A93ECE1FAE0B1E0BBBFB791BB2311F0E8
:10663C000E94225C1DE00E94FE611AE00E94FE6135
:10664C00DF91CF91E0E3F0E0EC0FFD1F10811870AB
:10665C00103010E011F008F01FEF112311F40C941E
:10666C005033CF93DF9318E0912A0BE71EE41A9373
:10667C000A93EDE2FAE0B1E0BBBFB791BB2311F096
:10668C000E94225C1DE00E94FE611AE00E94FE61E5
:10669C00DF91CF91E0E3F0E0EC0FFD1F108114705F
:1066AC00103010E011F008F01FEF112311F40C94CE
:1066BC007833CF93DF9318E0912A0BE71EE41A93FB
:1066CC000A93EEE3FAE0B1E0BBBFB791BB2311F044
:1066DC000E94225C1DE00E94FE611AE00E94FE6195
:1066EC00DF91CF91E0E3F0E0EC0FFD1F1081127011
:1066FC00103010E011F008F01FEF112311F40C947E
:10670C00A033CF93DF9318E0912A0BE71EE41A9382
:10671C000A93EFE4FAE0B1E0BBBFB791BB2311F0F1
:10672C000E94225C1DE00E94FE611AE00E94FE6144
:10673C00DF91CF91CF93DF9310E01A936197FE0115
:10674C00EF93FF933196FA93EA9310E11A9317EFB4
:10675C0091221FEB9122E4E6FAE0B1E0BBBFB791C6
:10676C00BB2311F00E94225C10E11F9318810F9142
:10677C00011B102FFF91EF91108323960E94C62CC2
:10678C00DF91CF910C940B34CF93DF9310E01A93DD
:10679C006197FE01EF93FF933196FA93EA9310E120
:1067AC001A9317EF91221FEB9122E4E7FAE0B1E084
:1067BC00BBBFB791BB2311F00E94225C10E11F9369
:1067CC0018810F91011B102FFF91EF9110832396CD
:1067DC000E94C62CDF91CF91CF93DF9318E0912AC2
:1067EC000BE71EE41A930A93EDE7FAE0B1E0BBBFA6
:1067FC00B791BB2311F00E94225C1DE00E94FE6148
:10680C001AE00E94FE61DF91CF9113E008EE0E9426
:10681C00295BCF93DF9310E01A936197FE01EF93FE
:10682C00FF933196FA93EA9310E11A9317EF9122A2
:10683C001FEB9122EDE8FAE0B1E0BBBFB791BB23AF
:10684C0011F00E94225C10E11F9318810F91011B23
:10685C00102FFF91EF91108323960E94C62CDF918D
:10686C00CF9111E004EF0E94295B10E0E0E3F0E02F
:10687C00EC0FFD1F1083CF93DF9318E0912A0BE7E9
:10688C001EE41A930A931DE00E94FE611AE00E9416
:10689C00FE61DF91CF91CF93DF9318E0912A0BE744
:1068AC001EE41A930A93EDE9FAE0B1E0BBBFB7918D
:1068BC00BB2311F00E94225C1DE00E94FE611AE0D5
:1068CC000E94FE61DF91CF91FE01F796FA93EA9355
:1068DC0011E0108317E31A931081088101171FEF41
:1068EC0008F01127112311F00C94E93410E0EEE3B9
:1068FC00F0E0EC0FFD1F10830E948563102FEBE37B
:10690C00F0E0EC0FFD1F1083CF93DF93EAE3F0E090
:10691C00EC0FFD1F10811A93ECE3F0E0EC0FFD1F60
:10692C0010811A930E94C907DF91CF91103010E0AB
:10693C0009F41FEF112311F40C94A934FE01F39602
:10694C00108113951083CF93DF93EAE3F0E0EC0F03
:10695C00FD1F10811A93FE01FF968F011A930A9363
:10696C000E94F307DF91CF91103010E009F41FEF74
:10697C00112311F40C94C734FE01F3961081139576
:10698C001083EBE3F0E0EC0FFD1F10811F93EEE39F
:10699C00F0E0EC0FFD1F10810F91011710E009F0D2
:1069AC001FEF112311F40C94E034FE01F3961081C7
:1069BC0013951083E981FA811081139510831123AB
:1069CC0011F00C9473342396E0E3F0E0EC0FFD1F10
:1069DC001081103010E011F008F01FEF112311F4AA
:1069EC000C943B35CF93DF9318E0912A0BE71EE410
:1069FC001A930A93EEEBFAE0B1E0BBBFB791BB235D
:106A0C0011F00E94225C1DE00E94FE611AE00E94BF
:106A1C00FE61DF91CF91CF93DF9310E01A936197D2
:106A2C00FE01EF93FF933196FA93EA9310E11A93D8
:106A3C0017EF91221FEB9122E8EDFAE0B1E0BBBF1A
:106A4C00B791BB2311F00E94225C10E11F931881B7
:106A5C000F91011B102FFF91EF91108323960E9431
:106A6C00C62CDF91CF910C947C35CF93DF9318E03B
:106A7C00912A0BE71EE41A930A93E8EEFAE0B1E0D0
:106A8C00BBBFB791BB2311F00E94225C1DE00E949A
:106A9C00FE611AE00E94FE61DF91CF91CF93DF93EC
:106AAC0010E01A936197FE01EF93FF933196FA93DE
:106ABC00EA9310E11A9317EF91221FEB9122EEEF5C
:106ACC00FAE0B1E0BBBFB791BB2311F00E94225C8E
:106ADC0010E11F9318810F91011B102FFF91EF9163
:106AEC00108323960E94C62CDF91CF9110E0E0E337
:106AFC00F0E0EC0FFD1F1083FE01B99613E010833C
:106B0C00FE01B996319613E01083FE01B9963296C8
:106B1C0013E01083FE01B996339613E01083CF93E4
:106B2C00DF93FE01B996249724E030E0DE010E9449
:106B3C00425B0E940D03DF91CF91103010E009F4FD
:106B4C001FEF112311F40C94B035FE01F096108157
:106B5C0013951083CF93DF93FE01B2968F011A9396
:106B6C000A930E94C300DF91CF91103010E009F41A
:106B7C001FEF112311F40C94C835FE01F09610810F
:106B8C0013951083FE01B996EF93FF93FE01B29615
:106B9C00EF93FF9324E030E0FF91EF91BF91AF9121
:106BAC000E94495B109510E009F01FEF112311F4BE
:106BBC000C94E535FE01F096108113951083FE01BF
:106BCC00BD961BE01083FE01BD9631961BE0108331
:106BDC00FE01BD96329617E31083CF93DF93FE012F
:106BEC00BD96239723E030E0DE010E94425B0E94B9
:106BFC00D602DF91CF91103010E009F41FEF112372
:106C0C0011F40C940E36FE01F0961081139510833E
:106C1C00FE01F796FA93EA9310E010831AE01A93A8
:106C2C001081088101171FEF08F01127112311F0B3
:106C3C000C948136CF93DF93FE0174968F011A93D7
:106C4C000A930E940507DF91CF91103010E009F4F0
:106C5C001FEF112311F40C943836FE01F3961081BA
:106C6C0013951083FE017496EF93FF933196FA936C
:106C7C00EA9310E11A9317EF91221FEB9122FE0178
:106C8C0077960E942A5C1DE00E94FE6110E11F9322
:106C9C0018810F91011B102FFF91EF9110832396F8
:106CAC00CF93DF9318E0912A0BE71EE41A930A9313
:106CBC00FE0176960E942A5CDF91CF9111E004EFE1
:106CCC00F8941093FD080093FC0810E41093F90855
:106CDC00F2011091FE080581101711F40E94B65AAA
:106CEC0097FC7894E981FA81108113951083112314
:106CFC0011F00C9417362396CF93DF93FE01B696C2
:106D0C008F011A930A930E946300DF91CF91103088
:106D1C0010E009F41FEF112311F40C949A36FE01C4
:106D2C00F096108113951083FE01B69610811B30DE
:106D3C0010E009F01FEF1F93FE01B69631961081FB
:106D4C001C3010E009F01FEF0F91102B1F93FE0168
:106D5C00B69632961081163031F020F4153010F0C2
:106D6C00442701C041E010E009F41FEF10950F918A
:106D7C00102B112311F40C94C836FE01F0961081DF
:106D8C0013951083CF93DF9318E0912A0BE71EE441
:106D9C001A930A931DE00E94FE611AE00E94FE61A4
:106DAC00DF91CF91E0E3F0E0EC0FFD1F108110308C
:106DBC0010E011F008F01FEF112311F40C94293797
:106DCC00CF93DF9318E0912A0BE71EE41A930A93F2
:106DDC00ECE0FBE0B1E0BBBFB791BB2311F00E942C
:106DEC00225C1DE00E94FE611AE00E94FE61DF91B0
:106DFC00CF91CF93DF9310E01A936197FE01EF933D
:106E0C00FF933196FA93EA9310E11A9317EF9122BC
:106E1C001FEB9122E8E2FBE0B1E0BBBFB791BB23D3
:106E2C0011F00E94225C10E11F9318810F91011B3D
:106E3C00102FFF91EF91108323960E94C62CDF91A7
:106E4C00CF910C946A37CF93DF9318E0912A0BE71C
:106E5C001EE41A930A93E8E3FBE0B1E0BBBFB791E1
:106E6C00BB2311F00E94225C1DE00E94FE611AE01F
:106E7C000E94FE61DF91CF91CF93DF9310E01A93C4
:106E8C006197FE01EF93FF933196FA93EA9310E129
:106E9C001A9317EF91221FEB9122E0E5FBE0B1E092
:106EAC00BBBFB791BB2311F00E94225C10E11F9372
:106EBC0018810F91011B102FFF91EF9110832396D6
:106ECC000E94C62CDF91CF9113E008EE0E94295B43
:106EDC00CF93DF9310E01A936197FE01EF93FF932A
:106EEC003196FA93EA9310E11A9317EF91221FEB64
:106EFC009122EEE5FBE0B1E0BBBFB791BB2311F0F3
:106F0C000E94225C10E11F9318810F91011B102F1E
:106F1C00FF91EF91108323960E94C62CDF91CF91A5
:106F2C0010E0E0E3F0E0EC0FFD1F108310E000E058
:106F3C00E1E3F0E0EC0FFD1F01931083CF93DF939F
:106F4C0018E0912A0BE71EE41A930A931DE00E94A5
:106F5C00FE611AE00E94FE61DF91CF91CF93DF9327
:106F6C0018E0912A0BE71EE41A930A93EEE5FBE076
:106F7C00B1E0BBBFB791BB2311F00E94225C1DE0B6
:106F8C000E94FE611AE00E94FE61DF91CF9110E039
:106F9C00EBE3F0E0EC0FFD1F10830E948563102FD4
:106FAC00E8E3F0E0EC0FFD1F1083E1E3F0E0EC0F01
:106FBC00FD1F019111910F931F93E8E3F0E0EC0F8B
:106FCC00FD1F1081012F11273F912F91020F131FCD
:106FDC00E1E3F0E0EC0FFD1F01931083E1E3F0E03F
:106FEC00EC0FFD1F01911191103809F4003010E0E5
:106FFC0011F008F01FEF112311F40C940D3810E868
:10700C0000E0E1E3F0E0EC0FFD1F01931083CF9360
:10701C00DF9310E01A93E2E3F0E0EC0FFD1F019117
:10702C0011911A930A93EBE3F0E0EC0FFD1F108122
:10703C001A930E941C2BDF91CF91103010E009F4B1
:10704C001FEF112311F40C943038FE01F0961081CF
:10705C0013951083CF93DF9310E01A93E2E3F0E0E3
:10706C00EC0FFD1F019111911A930A93FE01FE96EC
:10707C008F011A930A930E94E32ADF91CF9110306B
:10708C0010E009F41FEF112311F40C945238FE0197
:10709C00F096108113951083E8E3F0E0EC0FFD1FE0
:1070AC0010811F93EBE3F0E0EC0FFD1F10810F91AB
:1070BC00011710E009F01FEF112311F40C946B3839
:1070CC00FE01F096108113951083E1E3F0E0EC0FD4
:1070DC00FD1F01911191103809F4003010E009F4F2
:1070EC001FEF112311F40C94CD37E0E3F0E0EC0F1B
:1070FC00FD1F1081103010E011F008F01FEF11236C
:10710C0011F40C94CC38CF93DF9318E0912A0BE751
:10711C001EE41A930A93E0E7FBE0B1E0BBBFB79122
:10712C00BB2311F00E94225C1DE00E94FE611AE05C
:10713C000E94FE61DF91CF91CF93DF9310E01A9301
:10714C006197FE01EF93FF933196FA93EA9310E166
:10715C001A9317EF91221FEB9122ECE8FBE0B1E0C0
:10716C00BBBFB791BB2311F00E94225C10E11F93AF
:10717C0018810F91011B102FFF91EF911083239613
:10718C000E94C62CDF91CF910C940D39CF93DF93D5
:10719C0018E0912A0BE71EE41A930A93EAE9FBE044
:1071AC00B1E0BBBFB791BB2311F00E94225C1DE084
:1071BC000E94FE611AE00E94FE61DF91CF91CF9395
:1071CC00DF9310E01A936197FE01EF93FF933196D2
:1071DC00FA93EA9310E11A9317EF91221FEB912285
:1071EC00E2EBFBE0B1E0BBBFB791BB2311F00E9417
:1071FC00225C10E11F9318810F91011B102FFF913E
:10720C00EF91108323960E94C62CDF91CF91CF93E0
:10721C00DF9318E0912A0BE71EE41A930A931DE002
:10722C000E94FE611AE00E94FE61DF91CF91CF9324
:10723C00DF9318E0912A0BE71EE41A930A93EEEB06
:10724C00FBE0B1E0BBBFB791BB2311F00E94225C05
:10725C001DE00E94FE611AE00E94FE61DF91CF9159
:10726C00CF93DF9318E0912A0BE71EE41A930A934D
:10727C00E0EEFBE0B1E0BBBFB791BB2311F00E9485
:10728C00225C1DE00E94FE611AE00E94FE61DF910B
:10729C00CF91CF93DF9318E0912A0BE71EE41A935A
:1072AC000A93ECEFFBE0B1E0BBBFB791BB2311F04D
:1072BC000E94225C1DE00E94FE611AE00E94FE61A9
:1072CC00DF91CF91CF93DF93FE0171968F011A93CB
:1072DC000A9311E01A930E94700ADF91CF91CF9319
:1072EC00DF9318E0912A0BE71EE41A930A931DE032
:1072FC000E94FE611AE00E94FE61DF91CF91CF9354
:10730C00DF9310E01A936197FE01EF93FF93319690
:10731C00FA93EA9310E11A9317EF91221FEB912243
:10732C00EFE0FCE0B1E0BBBFB791BB2311F00E94D2
:10733C00225C10E11F9318810F91011B102FFF91FC
:10734C00EF91108323960E94C62CDF91CF91CF939F
:10735C00DF9310E004E31A930A9310E81A9310E8F1
:10736C001A930E94A22DDF91CF91CF93DF9310E05F
:10737C0005E31A930A9310E81A9310E81A930E94E3
:10738C00A22DDF91CF91FE01719610E11083FE01C9
:10739C00F796FA93EA9311E0108310E11A93108197
:1073AC00088101171FEF08F01127112311F00C941D
:1073BC00093A0E948563102FEBE3F0E0EC0FFD1F00
:1073CC001083FE017496EF93FF93EAE3F0E0EC0F69
:1073DC00FD1F1081FF91EF91012F1127E00FF11F7D
:1073EC00EF93FF93EBE3F0E0EC0FFD1F1081FF91A7
:1073FC00EF911193E981FA81108113951083112378
:10740C0011F00C94D6392396CF93DF9318E0912A80
:10741C0002EC1EE41A930A93FE0173960E942A5CF6
:10742C001DE00E94FE61DF91CF911FEFE3E3F0E0DE
:10743C00EC0FFD1F108311E0E7E3F0E0EC0FFD1FF4
:10744C00108313E008EE9801E7E3F2E010811123BA
:10745C0029F40E94C75AE7E3F2E01081112309F0E6
:10746C001FEF112311F40C947C3A0E949E4EE4E31E
:10747C00F0E0EC0FFD1F1083E4E3F0E0EC0FFD1FD8
:10748C0010811D3010E009F01FEF112311F40C9442
:10749C006E3AFE01EF93FF93E7E3F0E0EC0FFD1F74
:1074AC001081FF91EF91012F1127E00FF11FEF9346
:1074BC00FF93E4E3F0E0EC0FFD1F1081FF91EF91DF
:1074CC001193FE01F7961081139510830C947A3A60
:1074DC00FE01EF93FF93E7E3F0E0EC0FFD1F10814B
:1074EC001150FF91EF9111930C94823A10E0E3E369
:1074FC00F0E0EC0FFD1F1083E4E3F0E0EC0FFD1F58
:10750C0010811D3010E009F41FEF1F93E3E3F0E04E
:10751C00EC0FFD1F1081103010E009F41FEF0F91DC
:10752C00102B112311F40C94273AFE01EF93FF93C7
:10753C00FE017196BF91AF91E89494F80E94355D6D
:10754C0010E009F41FEF1F93E3E3F0E0EC0FFD1FD5
:10755C0010811F3F10E009F41FEF0F91102311232E
:10756C0011F40C94FC3ACF93DF9318E0912A0BE7BB
:10757C001EE41A930A93EFE1FCE0B1E0BBBFB791B4
:10758C00BB2311F00E94225C1DE00E94FE611AE0F8
:10759C000E94FE61DF91CF91CF93DF9310E01A939D
:1075AC006197FE01EF93FF933196FA93EA9310E102
:1075BC001A9317EF91221FEB9122E4E3FCE0B1E068
:1075CC00BBBFB791BB2311F00E94225C10E11F934B
:1075DC0018810F91011B102FFF91EF9110832396AF
:1075EC000E94C62CDF91CF910C943D3BCF93DF933F
:1075FC0018E0912A0BE71EE41A930A93E1E4FCE0ED
:10760C00B1E0BBBFB791BB2311F00E94225C1DE01F
:10761C000E94FE611AE00E94FE61DF91CF91CF9330
:10762C00DF9310E01A936197FE01EF93FF9331966D
:10763C00FA93EA9310E11A9317EF91221FEB912220
:10764C00EAE5FCE0B1E0BBBFB791BB2311F00E94AF
:10765C00225C10E11F9318810F91011B102FFF91D9
:10766C00EF91108323960E94C62CDF91CF91CF937C
:10767C00DF9318E0912A0BE71EE41A930A93E9E6CC
:10768C00FCE0B1E0BBBFB791BB2311F00E94225CC0
:10769C001DE00E94FE611AE00E94FE61DF91CF9115
:1076AC00CF93DF93FE0171968F011A930A9311E029
:1076BC001A930E94700ADF91CF91CF93DF9318E059
:1076CC00912A0BE71EE41A930A931DE00E94FE61B7
:1076DC001AE00E94FE61DF91CF91CF93DF9310E00F
:1076EC0005E31A930A9310E81A9310E01A930E9478
:1076FC00A22DDF91CF91FE01719610E11083FE0156
:10770C00F796FA93EA9311E0108310E11A93108123
:10771C00088101171FEF08F01127112311F00C94A9
:10772C00C13B0E948563102FEBE3F0E0EC0FFD1FD3
:10773C001083FE017496EF93FF93EAE3F0E0EC0FF5
:10774C00FD1F1081FF91EF91012F1127E00FF11F09
:10775C00EF93FF93EBE3F0E0EC0FFD1F1081FF9133
:10776C00EF911193E981FA81108113951083112304
:10777C0011F00C948E3B2396CF93DF9318E0912A53
:10778C0002EC1EE41A930A93FE0173960E942A5C83
:10779C001DE00E94FE61DF91CF911FEFE3E3F0E06B
:1077AC00EC0FFD1F108311E0E7E3F0E0EC0FFD1F81
:1077BC00108313E008EE9801E7E3F2E01081112347
:1077CC0029F40E94C75AE7E3F2E01081112309F073
:1077DC001FEF112311F40C94343C0E949E4EE4E3F1
:1077EC00F0E0EC0FFD1F1083E4E3F0E0EC0FFD1F65
:1077FC0010811D3010E009F01FEF112311F40C94CF
:10780C00263CFE01EF93FF93E7E3F0E0EC0FFD1F46
:10781C001081FF91EF91012F1127E00FF11FEF93D2
:10782C00FF93E4E3F0E0EC0FFD1F1081FF91EF916B
:10783C001193FE01F7961081139510830C94323C32
:10784C00FE01EF93FF93E7E3F0E0EC0FFD1F1081D7
:10785C001150FF91EF9111930C943A3C10E0E3E33B
:10786C00F0E0EC0FFD1F1083E4E3F0E0EC0FFD1FE4
:10787C0010811D3010E009F41FEF1F93E3E3F0E0DB
:10788C00EC0FFD1F1081103010E009F41FEF0F9169
:10789C00102B112311F40C94DF3BFE01EF93FF939B
:1078AC00FE017196BF91AF91E89494F80E94355DFA
:1078BC0010E009F41FEF1F93E3E3F0E0EC0FFD1F62
:1078CC0010811F3F10E009F41FEF0F9110231123BB
:1078DC0011F40C94B43CCF93DF9318E0912A0BE78E
:1078EC001EE41A930A93ECE8FCE0B1E0BBBFB7913D
:1078FC00BB2311F00E94225C1DE00E94FE611AE085
:10790C000E94FE61DF91CF91CF93DF9310E01A9329
:10791C006197FE01EF93FF933196FA93EA9310E18E
:10792C001A9317EF91221FEB9122E1EAFCE0B1E0F0
:10793C00BBBFB791BB2311F00E94225C10E11F93D7
:10794C0018810F91011B102FFF91EF91108323963B
:10795C000E94C62CDF91CF910C94F53CCF93DF9312
:10796C0018E0912A0BE71EE41A930A93EEEAFCE066
:10797C00B1E0BBBFB791BB2311F00E94225C1DE0AC
:10798C000E94FE611AE00E94FE61DF91CF91CF93BD
:10799C00DF9310E01A936197FE01EF93FF933196FA
:1079AC00FA93EA9310E11A9317EF91221FEB9122AD
:1079BC00E7ECFCE0B1E0BBBFB791BB2311F00E9438
:1079CC00225C10E11F9318810F91011B102FFF9166
:1079DC00EF91108323960E94C62CDF91CF9113E078
:1079EC0008EE0E94295BCF93DF9310E01A93619706
:1079FC00FE01EF93FF933196FA93EA9310E11A93F9
:107A0C0017EF91221FEB9122E6EDFCE0B1E0BBBF3A
:107A1C00B791BB2311F00E94225C10E11F931881D7
:107A2C000F91011B102FFF91EF91108323960E9451
:107A3C00C62CDF91CF91CF93DF9318E0912A0BE7FF
:107A4C001EE41A930A93E2EEFCE0B1E0BBBFB791DF
:107A5C00BB2311F00E94225C1DE00E94FE611AE023
:107A6C000E94FE61DF91CF910895CF93DF93E5E4FF
:107A7C00F7E0FA93EA936097FE01EF93FF93319648
:107A8C00FA93EA931FE01A9317EF91221FEB9122BE
:107A9C00FE0175960E942A5C1FE01F9318810F91BE
:107AAC00011B102FFF91EF91108323960E944F58CA
:107ABC00DF91CF91112311F40C94693D1FEF0C94BD
:107ACC00903D0C948F3DCF93DF9318E0912A0BE7F8
:107ADC001EE41A930A93E5E0FDE0B1E0BBBFB79159
:107AEC00BB2311F00E94225CFE0132960E942A5C9C
:107AFC00E3E1FDE0B1E0BBBFB791BB2311F00E9405
:107B0C00225C1DE00E94FE611AE00E94FE61DF9182
:107B1C00CF9110E00895CF93DF9318E0912A0BE7F3
:107B2C001EE41A930A93EBE1FDE0B1E0BBBFB79101
:107B3C00BB2311F00E94225C1DE00E94FE611AE042
:107B4C000E94FE61DF91CF91CF93DF9318E0912AD1
:107B5C000BE71EE41A930A93E4E3FDE0B1E0BBBF2C
:107B6C00B791BB2311F00E94225C1DE00E94FE61C4
:107B7C001AE00E94FE61DF91CF91CF93DF9318E062
:107B8C00912A0BE71EE41A930A93EDE4FDE0B1E0B1
:107B9C00BBBFB791BB2311F00E94225C1DE00E9479
:107BAC00FE611AE00E94FE61DF91CF91CF93DF93CB
:107BBC0018E0912A0BE71EE41A930A93EDE6FDE018
:107BCC00B1E0BBBFB791BB2311F00E94225C1DE05A
:107BDC000E94FE611AE00E94FE61DF91CF91CF936B
:107BEC00DF9318E0912A0BE71EE41A930A93ECE852
:107BFC00FDE0B1E0BBBFB791BB2311F00E94225C4A
:107C0C001DE00E94FE611AE00E94FE61DF91CF919F
:107C1C00CF93DF9318E0912A0BE71EE41A930A9393
:107C2C00EFEBFDE0B1E0BBBFB791BB2311F00E94BD
:107C3C00225C1DE00E94FE611AE00E94FE61DF9151
:107C4C00CF91CF93DF9318E0912A0BE71EE41A93A0
:107C5C000A93EAEDFDE0B1E0BBBFB791BB2311F095
:107C6C000E94225C1DE00E94FE611AE00E94FE61EF
:107C7C00DF91CF91CF93DF9318E0912A0BE71EE4AD
:107C8C001A930A93E2E0FEE0B1E0BBBFB791BB23CD
:107C9C0011F00E94225C1DE00E94FE611AE00E941D
:107CAC00FE61DF91CF91CF93DF9318E0912A0BE720
:107CBC001EE41A930A93ECE2FEE0B1E0BBBFB7916D
:107CCC00BB2311F00E94225C1DE00E94FE611AE0B1
:107CDC000E94FE61DF91CF91CF93DF9318E0912A40
:107CEC000BE71EE41A930A93EDE4FEE0B1E0BBBF90
:107CFC00B791BB2311F00E94225C1DE00E94FE6133
:107D0C001AE00E94FE61DF91CF91CF93DF9318E0D0
:107D1C00912A0BE71EE41A930A93E8E7FEE0B1E020
:107D2C00BBBFB791BB2311F00E94225C1DE00E94E7
:107D3C00FE611AE00E94FE61DF91CF91CF93DF9339
:107D4C0018E0912A0BE71EE41A930A93E0EAFEE08E
:107D5C00B1E0BBBFB791BB2311F00E94225C1DE0C8
:107D6C000E94FE611AE00E94FE61DF91CF9108959E
:107D7C0020E030E0EBE9F4E01081112329F40E94BB
:107D8C00C75AEBE9F4E01081112309F01FEFABE9BE
:107D9C00B4E042EA54E00E941E64F8941093270861
:107DAC0097FC789410912708103011F00C94E23E57
:107DBC000E94913D0C944249113011F00C948B3F70
:107DCC00CF93DF9318E0912A0BE71EE41A930A93E2
:107DDC001DE00E94FE611AE00E94FE61DF91CF91CE
:107DEC00CF93DF9318E0912A0BE71EE41A930A93C2
:107DFC00E6EDFEE0B1E0BBBFB791BB2311F00E94F2
:107E0C00225CDF91CF91CF93DF93E2E3F8E08F0117
:107E1C001A930A9310E11A930E94700ADF91CF9182
:107E2C00CF93DF9318E0912A0BE71EE41A930A9381
:107E3C001DE00E94FE611AE00E94FE61DF91CF916D
:107E4C00CF93DF936097FE01EF93FF933196FA93F4
:107E5C00EA931FE01A9317EF91221FEB9122E2E3B2
:107E6C00F8E0F8940E942A5C97FC78941FE01F932A
:107E7C0018810F91011B102FFF91EF911083239606
:107E8C000E942C58DF91CF91112311F40C94703F68
:107E9C00CF93DF9318E0912A0BE71EE41A930A9311
:107EAC00E2E3F8E0F8940E942A5C97FC7894E2EE06
:107EBC00FEE0B1E0BBBFB791BB2311F00E94225C86
:107ECC001DE00E94FE611AE00E94FE61DF91CF91DD
:107EDC000C94893FCF93DF9318E0912A0BE71EE4B3
:107EEC001A930A93EBEEFEE0B1E0BBBFB791BB2354
:107EFC0011F00E94225C1DE00E94FE611AE00E94BB
:107F0C00FE61DF91CF910C944249123011F00C9428
:107F1C003440CF93DF9318E0912A0BE71EE41A93B9
:107F2C000A931DE00E94FE611AE00E94FE61DF913F
:107F3C00CF91CF93DF9318E0912A0BE71EE41A93AD
:107F4C000A93E6EDFEE0B1E0BBBFB791BB2311F0A5
:107F5C000E94225CDF91CF91CF93DF93E2E3F8E0B4
:107F6C008F011A930A9310E11A930E94700ADF9101
:107F7C00CF91CF93DF9318E0912A0BE71EE41A936D
:107F8C000A931DE00E94FE611AE00E94FE61DF91DF
:107F9C00CF91CF93DF936097FE01EF93FF933196D0
:107FAC00FA93EA931FE01A9317EF91221FEB912299
:107FBC00E2E3F8E0F8940E942A5C97FC78941FE0C6
:107FCC001F9318810F91011B102FFF91EF911083BC
:107FDC0023960E944458DF91CF91112311F40C94F5
:107FEC001940CF93DF9318E0912A0BE71EE41A9304
:107FFC000A93E2E3F8E0F8940E942A5C97FC7894E8
:10800C00EEEFFEE0B1E0BBBFB791BB2311F00E94D5
:10801C00225C1DE00E94FE611AE00E94FE61DF916D
:10802C00CF910C943240CF93DF9318E0912A0BE759
:10803C001EE41A930A93E7E0FFE0B1E0BBBFB791EF
:10804C00BB2311F00E94225C1DE00E94FE611AE02D
:10805C000E94FE61DF91CF910C944249133011F0D4
:10806C000C941E41CF93DF9318E0912A0BE71EE48A
:10807C001A930A931DE00E94FE611AE00E94FE61B1
:10808C00DF91CF91CF93DF9318E0912A0BE71EE499
:10809C001A930A93E6EDFEE0B1E0BBBFB791BB23A8
:1080AC0011F00E94225CDF91CF91CF93DF93E2E33A
:1080BC00F8E08F011A930A9310E11A930E94700A48
:1080CC00DF91CF91CF93DF9318E0912A0BE71EE459
:1080DC001A930A931DE00E94FE611AE00E94FE6151
:1080EC00DF91CF91CF93DF936197FE01EF93FF93D5
:1080FC003196FA93EA9310E11A9317EF91221FEB42
:10810C009122E2E3F8E0F8940E942A5C97FC7894C0
:10811C0010E11F9318810F91011B102FFF91EF910C
:10812C00108323960E943B3DDF91CF91112311F4D4
:10813C000C941C41CF93DF9318E0912A0BE71EE4BB
:10814C001A930A93EEE5F8E0B1E0BBBFB791BB23FD
:10815C0011F00E94225C1DE00E94FE611AE00E9458
:10816C00FE61DF91CF910E944D4EF894109326083A
:10817C0097FC7894109126081D3010E009F41FEF3D
:10818C00112311F40C94CC400C940241CF93DF9347
:10819C0018E0912A0BE71EE41A930A931091260813
:1081AC000E94FE6197FC7894DF91CF91CF93DF937F
:1081BC0000914507109146071A930A93E6E2F8E0FE
:1081CC00FA93EA9310E001E01A930A930F931F932A
:1081DC000E943B5A1F910F9128813981021B131B5E
:1081EC00DF91CF91109126081D3010E009F41FEF9C
:1081FC00112311F40C94B940CF93DF93E5E4F7E02D
:10820C00FA93EA930E947D58DF91CF91CF93DF933D
:10821C0018E0912A0BE71EE41A930A931DE00E94C2
:10822C00FE611AE00E94FE61DF91CF910C944249ED
:10823C00143011F00C94D941CF93DF9318E0912AAC
:10824C000BE71EE41A930A931DE00E94FE611AE0EC
:10825C000E94FE61DF91CF91CF93DF9318E0912ABA
:10826C000BE71EE41A930A93E6EDFEE0B1E0BBBF08
:10827C00B791BB2311F00E94225CDF91CF91CF9379
:10828C00DF93E2E3F8E08F011A930A9310E11A935B
:10829C000E94700ADF91CF91CF93DF9318E0912A5F
:1082AC000BE71EE41A930A931DE00E94FE611AE08C
:1082BC000E94FE61DF91CF91CF93DF936197FE0116
:1082CC00EF93FF933196FA93EA9310E11A9317EF19
:1082DC0091221FEB9122E2E3F8E0F8940E942A5CD1
:1082EC0097FC789410E11F9318810F91011B102FAC
:1082FC00FF91EF91108323960E943B3DDF91CF912C
:10830C00112311F40C94D7410091450710914607A5
:10831C000E9431591095112311F40C94BD41CF9347
:10832C00DF9300914507109146071A930A93E6E2F2
:10833C00F8E0FA93EA9310E001E01A930A930E9492
:10834C00CC5908811981DF91CF91CF93DF9318E03D
:10835C00912A0BE71EE41A930A93109126080E94A7
:10836C00FE6197FC7894DF91CF910C948A41CF9366
:10837C00DF93E5E4F7E0FA93EA930E947D58DF91EE
:10838C00CF91CF93DF9318E0912A0BE71EE41A9359
:10839C000A931DE00E94FE611AE00E94FE61DF91CB
:1083AC00CF910C944249153011F00C948D43CF931E
:1083BC00DF9318E0912A0BE71EE41A930A931DE051
:1083CC000E94FE611AE00E94FE61DF91CF91CF9373
:1083DC00DF9318E0912A0BE71EE41A930A93E6ED5B
:1083EC00FEE0B1E0BBBFB791BB2311F00E94225C51
:1083FC00DF91CF91CF93DF93E2E3F8E08F011A93F3
:10840C000A9310E11A930E94700ADF91CF91CF93D7
:10841C00DF9318E0912A0BE71EE41A930A931DE0F0
:10842C000E94FE611AE00E94FE61DF91CF91CF9312
:10843C00DF9318E0912A0BE71EE41A930A93EAE102
:10844C00FFE0B1E0BBBFB791BB2311F00E94225CEF
:10845C00DF91CF91CF93DF930E949C09DF91CF9155
:10846C00012F112733272227F89400932A08109301
:10847C002B0820932C0830932D0897FC7894CF93DD
:10848C00DF9318E0912A0BE71EE41A930A931DE080
:10849C000E94FE611AE00E94FE61DF91CF91CF93A2
:1084AC00DF936197FE01EF93FF933196FA93EA9372
:1084BC0010E11A9317EF91221FEB9122E2E3F8E0FF
:1084CC00F8940E942A5C97FC789410E11F93188111
:1084DC000F91011B102FFF91EF91108323960E9497
:1084EC003B3DDF91CF91112311F40C948B43CF932F
:1084FC00DF9300914507109146071A930A9310E0F9
:10850C0001E01A930A93F89400912A0810912B0811
:10851C0020912C0830912D0897FC78943A932A934B
:10852C001A930A930E944A59DF91CF91F8940093C1
:10853C002E0810932F08209330083093310897FCA5
:10854C00789400914507109146070E9431591123E8
:10855C0011F40C94CA42CF93DF9318E0912A0BE7E5
:10856C001EE41A930A93E0E3FFE0B1E0BBBFB791BE
:10857C00BB2311F00E94225C1DE00E94FE611AE0F8
:10858C000E94FE61DF91CF91F89400912E0810911A
:10859C002F08209130083091310897FC78940F9374
:1085AC001F932F933F93F89400912A0810912B0856
:1085BC0020912C0830912D0897FC7894D801F90162
:1085CC003F912F911F910F913F1729F42E1719F4FA
:1085DC001B1709F40A1710E009F41FEF112311F40B
:1085EC000C945843CF93DF9318E0912A0BE71EE4C9
:1085FC001A930A93E4E3FFE0B1E0BBBFB791BB234E
:10860C0011F00E94225CF89400912E0810912F0812
:10861C00209130083091310897FC7894E89495F8C3
:10862C0050E040E0E0E20E94745C1DE00E94FE61BC
:10863C001AE00E94FE61DF91CF91009145071091E5
:10864C0046070E9431591095112311F40C9456438E
:10865C00CF93DF9300914507109146071A930A9325
:10866C00E6E2F8E0FA93EA9310E001E01A930A9339
:10867C000E94CC5908811981DF91CF91CF93DF9360
:10868C0018E0912A0BE71EE41A930A93109126081E
:10869C000E94FE6197FC7894DF91CF910C94234358
:1086AC000C947143CF93DF9318E0912A0BE71EE4EF
:1086BC001A930A93EDE3FFE0B1E0BBBFB791BB2384
:1086CC0011F00E94225C1DE00E94FE611AE00E94E3
:1086DC00FE61DF91CF91CF93DF93E5E4F7E0FA935E
:1086EC00EA930E947D58DF91CF91CF93DF9318E0EE
:1086FC00912A0BE71EE41A930A931DE00E94FE6177
:10870C001AE00E94FE61DF91CF910C944249163021
:10871C0011F00C949A44CF93DF9318E0912A0BE755
:10872C001EE41A930A931DE00E94FE611AE00E9457
:10873C00FE61DF91CF91CF93DF9318E0912A0BE785
:10874C001EE41A930A93E6EDFEE0B1E0BBBFB791CD
:10875C00BB2311F00E94225CDF91CF91CF93DF936A
:10876C00E2E3F8E08F011A930A9310E11A930E9446
:10877C00700ADF91CF91CF93DF936197FE01EF9356
:10878C00FF933196FA93EA9310E11A9317EF912223
:10879C001FEB9122E2E3F8E0F8940E942A5C97FC2C
:1087AC00789410E11F9318810F91011B102FFF91EA
:1087BC00EF91108323960E943B3DDF91CF911123C3
:1087CC0011F40C949844CF93DF9318E0912A0BE7A3
:1087DC001EE41A930A931DE00E94FE611AE00E94A7
:1087EC00FE61DF91CF91CF93DF9318E0912A0BE7D5
:1087FC001EE41A930A93E2E3F8E0F8940E942A5CD0
:10880C0097FC7894EBE4FFE0B1E0BBBFB791BB23DE
:10881C0011F00E94225C1DE00E94FE611AE00E9491
:10882C00FE61DF91CF91F89410E01093280897FC2B
:10883C00789400914507109146070E943159109584
:10884C00112311F40C947E44CF93DF9300914507D0
:10885C00109146071A930A93E9E2F8E0FA93EA9327
:10886C0010E001E01A930A930E94CC5908811981F7
:10887C00DF91CF91CF93DF9318E0912A0BE71EE4A1
:10888C001A930A9310912908412F0E94505D10E20F
:10889C000E94FE61DF91CF91109128081F3010E0EB
:1088AC0009F41FEF112311F40C947444CF93DF934C
:1088BC0018E0912A0BE71EE41A930A931DE00E941C
:1088CC00FE611AE00E94FE61DF91CF91F89410E0F6
:1088DC001093280897FC78940C947C44F89410918D
:1088EC00280813951093280897FC78940C941F442F
:1088FC00CF93DF93E5E4F7E0FA93EA930E947D5877
:10890C00DF91CF91CF93DF9318E0912A0BE71EE410
:10891C001A930A931DE00E94FE611AE00E94FE6108
:10892C00DF91CF910C944249173011F00C944045D3
:10893C00CF93DF9318E0912A0BE71EE41A930A9366
:10894C001DE00E94FE611AE00E94FE61DF91CF9152
:10895C00CF93DF93E2E3F8E0FA93EA936097FE019A
:10896C00EF93FF933196FA93EA931FE01A9317EF64
:10897C0091221FEB9122E5E5FFE0B1E0BBBFB7917F
:10898C00BB2311F00E94225C1FE01F9318810F91F2
:10899C00011B102FFF91EF91108323960E94AA5870
:1089AC00DF91CF91112311F40C942545CF93DF93D4
:1089BC0018E0912A0BE71EE41A930A93E2E3F8E01D
:1089CC00F8940E942A5C97FC78941DE00E94FE614A
:1089DC001AE00E94FE61DF91CF91CF93DF93E2E327
:1089EC00F8E0FA93EA930E94BD58DF91CF911123DE
:1089FC0011F40C942345CF93DF9318E0912A0BE7E5
:108A0C001EE41A930A93E2E3F8E0F8940E942A5CBD
:108A1C0097FC7894E9E5FFE0B1E0BBBFB791BB23CD
:108A2C0011F00E94225C1DE00E94FE611AE00E947F
:108A3C00FE61DF91CF910C94F3440C943E45CF939F
:108A4C00DF9318E0912A0BE71EE41A930A93EDE5E5
:108A5C00FFE0B1E0BBBFB791BB2311F00E94225CD9
:108A6C001DE00E94FE611AE00E94FE61DF91CF9131
:108A7C000C944249183011F00C948C45CF93DF9331
:108A8C0018E0912A0BE71EE41A930A931DE00E944A
:108A9C00FE611AE00E94FE61DF91CF91CF93DF93CC
:108AAC0018E0912A0BE71EE41A930A93ECE6FFE018
:108ABC00B1E0BBBFB791BB2311F00E94225CDF91E8
:108ACC00CF91CF93DF9318E0912A0BE71EE41A9312
:108ADC000A9311E40E940559E89495F850E040E09F
:108AEC00E0E20E94AB5CEEE7FFE0B1E0BBBFB79108
:108AFC00BB2311F00E94225C1DE00E94FE611AE073
:108B0C000E94FE61DF91CF910C944249193011F013
:108B1C000C94DD45CF93DF9318E0912A0BE71EE40C
:108B2C001A930A931DE00E94FE611AE00E94FE61F6
:108B3C00DF91CF9111E40E948D4F112311F40C940D
:108B4C00C245CF93DF9318E0912A0BE71EE41A93EA
:108B5C000A93E6E8FFE0B1E0BBBFB791BB2311F08D
:108B6C000E94225C1DE00E94FE611AE00E94FE61E0
:108B7C00DF91CF910C94DB45CF93DF9318E0912AD2
:108B8C000BE71EE41A930A93E2E9FFE0B1E0BBBFE6
:108B9C00B791BB2311F00E94225C1DE00E94FE6184
:108BAC001AE00E94FE61DF91CF910C9442491A3079
:108BBC0011F00C942246CF93DF9318E0912A0BE727
:108BCC001EE41A930A931DE00E94FE611AE00E94B3
:108BDC00FE61DF91CF91CF93DF9318E0912A0BE7E1
:108BEC001EE41A930A93E0EAFFE0B1E0BBBFB79131
:108BFC00BB2311F00E94225CDF91CF91CF93DF93C6
:108C0C00E2E3F8E08F011A930A9310E11A930E94A1
:108C1C00700ADF91CF91E2E3F8E0F8940E94B65F1E
:108C2C0097FC7894009347071093480720934907C3
:108C3C0030934A070C9442491B3011F00C94D646E1
:108C4C00CF93DF9318E0912A0BE71EE41A930A9353
:108C5C001DE00E94FE611AE00E94FE61DF91CF913F
:108C6C00CF93DF9318E0912A0BE71EE41A930A9333
:108C7C00E1EBFFE0B1E0BBBFB791BB2311F00E9469
:108C8C00225C0091470710914807209149073091C9
:108C9C004A07B4E0A2E0E0E20E94CA6016E50E9436
:108CAC00FE611DE00E94FE611AE00E94FE61DF91F0
:108CBC00CF91E8E2F8E0FA93EA9311E0108318E020
:108CCC001A931081088101171FEF08F01127112347
:108CDC0011F00C94D346CF93DF9318E0912A0BE755
:108CEC001EE41A930A93E9EBFFE0B1E0BBBFB79126
:108CFC00BB2311F00E94225C1091280850E040E048
:108D0C00E0E20E94345CE6E5F0E0B1E0BBBFB79175
:108D1C00BB2311F00E94225C009147071091480779
:108D2C002091490730914A07A801B901A0E0B0ECA5
:108D3C00EFE7F4E4E89491F80E948A5E0F931F9396
:108D4C002F933F93109128080E94DB630F7F1370C1
:108D5C0033272227E89495F8E89491F80E94DE5D79
:108D6C00E89491F80E940E5EB4E0A2E0E0E20E946A
:108D7C00CA6016E50E94FE611DE00E94FE611AE0C9
:108D8C000E94FE61DF91CF91E981FA8110811395E8
:108D9C001083112311F00C94684623960C944249CD
:108DAC001C3011F00C943447CF93DF9318E0912AC8
:108DBC000BE71EE41A930A931DE00E94FE611AE071
:108DCC000E94FE61DF91CF91CF93DF9318E0912A3F
:108DDC000BE71EE41A930A93EDEBFFE0B1E0BBBF87
:108DEC00B791BB2311F00E94225CDF91CF91CF93FE
:108DFC00DF93E2E3F8E08F011A930A9310E11A93E0
:108E0C000E94700ADF91CF910E94932DCF93DF9334
:108E1C0010E01A936197FE01EF93FF933196FA934A
:108E2C00EA9310E11A9317EF91221FEB9122E2E3E0
:108E3C00F8E0F8940E942A5C97FC789410E11F9358
:108E4C0018810F91011B102FFF91EF911083239626
:108E5C000E94C62CDF91CF910C9442491D3011F029
:108E6C000C945047CF93DF9318E0912A0BE71EE444
:108E7C001A930A931DE00E94FE611AE00E94FE61A3
:108E8C00DF91CF91CF93DF930E94E92DDF91CF91AA
:108E9C000C9442491E3011F00C944548CF93DF934B
:108EAC0018E0912A0BE71EE41A930A931DE00E9426
:108EBC00FE611AE00E94FE61DF91CF91CF93DF93A8
:108ECC0018E0912A0BE71EE41A930A93ECECFFE0EE
:108EDC00B1E0BBBFB791BB2311F00E94225CDF91C4
:108EEC00CF91CF93DF93E3E4F8E08F011A930A93C9
:108EFC0011E01A930E94700ADF91CF91CF93DF9308
:108F0C0018E0912A0BE71EE41A930A931DE00E94C5
:108F1C00FE611AE00E94FE61DF91CF91CF93DF9347
:108F2C0018E0912A0BE71EE41A930A93E3EEFFE094
:108F3C00B1E0BBBFB791BB2311F00E94225CDF9163
:108F4C00CF91CF93DF930E94E908DF91CF91F894F2
:108F5C001093290897FC7894E3E4F8E03196EF93AA
:108F6C00FF93E3E4F8E031961081113618F01B37CB
:108F7C0008F41052F894FF91EF91119397FC7894A8
:108F8C00E3E4F8E031961081163431F020F411341A
:108F9C0010F0442701C041E010E009F41FEF112349
:108FAC0011F40C944348E3E4F8E031961081113449
:108FBC0011F00C94EE47CF93DF9310E01A931091BD
:108FCC0029081A930E94382CDF91CF910C944348B6
:108FDC00123411F00C94FF47CF93DF9311E01A93E6
:108FEC00109129081A930E94382CDF91CF910C9480
:108FFC004348133411F00C941048CF93DF9312E0D4
:10900C001A93109129081A930E94382CDF91CF9152
:10901C000C944348143411F00C942148CF93DF93F3
:10902C0013E01A93109129081A930E94382CDF919F
:10903C00CF910C944348153411F00C943248CF93D3
:10904C00DF9314E01A93109129081A930E94382C7C
:10905C00DF91CF910C944348163411F00C94434893
:10906C00CF93DF9315E01A93109129081A930E945D
:10907C00382CDF91CF910C9443480C9442491F300B
:10908C0011F00C944249CF93DF9318E0912A0BE72F
:10909C001EE41A930A931DE00E94FE611AE00E94DE
:1090AC00FE61DF91CF91CF93DF9318E0912A0BE70C
:1090BC001EE41A930A93E4EFFFE0B1E0BBBFB79153
:1090CC00BB2311F00E94225CDF91CF91CF93DF93F1
:1090DC00E3E4F8E08F011A930A9311E01A930E94CB
:1090EC00700ADF91CF91E3E4F8E03196EF93FF93B0
:1090FC00E3E4F8E031961081113618F01B3708F4D0
:10910C001052F894FF91EF91119397FC7894E3E44B
:10911C00F8E031961081163431F020F4113410F04F
:10912C00442701C041E010E009F41FEF112311F4B2
:10913C000C944049E3E4F8E031961081113411F0BD
:10914C000C94B648CF93DF9310E01A9318E009E221
:10915C001A930A930E945C2CDF91CF910C941049C6
:10916C00123411F00C94C848CF93DF9311E01A938A
:10917C0018E009E21A930A930E945C2CDF91CF91BC
:10918C000C941049133411F00C94DA48CF93DF93FC
:10919C0012E01A9318E009E21A930A930E945C2CCD
:1091AC00DF91CF910C941049143411F00C94EC48CD
:1091BC00CF93DF9313E01A9318E009E21A930A9302
:1091CC000E945C2CDF91CF910C941049153411F056
:1091DC000C94FE48CF93DF9314E01A9318E009E245
:1091EC001A930A930E945C2CDF91CF910C94104936
:1091FC00163411F00C941049CF93DF9315E01A93A9
:10920C0018E009E21A930A930E945C2CDF91CF912B
:10921C000C941049CF93DF9318E0912A0BE71EE4CE
:10922C001A930A931DE00E94FE611AE00E94FE61EF
:10923C00DF91CF91CF93DF9318E0912A0BE71EE4D7
:10924C001A930A93EAE0F0E1B1E0BBBFB791BB23FC
:10925C0011F00E94225C1091290850E040E0E0E2FD
:10926C000E94345C1DE00E94FE611AE00E94FE61C7
:10927C00DF91CF910C94424910E11093E9080C94C2
:10928C00BE3E00E010E020EA30E400934707109364
:10929C0048072093490730934A07CF93DF93E6E4BE
:1092AC00F6E08F011A930A931FE01A930E942C0880
:1092BC00DF91CF91CF93DF9311E01A930E94482B4B
:1092CC00DF91CF910E94205810E8912A7894F8945D
:1092DC00112712BF16B7117016BF10E8912A789497
:1092EC000E94932DCF93DF9310E01A936197FE01A8
:1092FC00EF93FF933196FA93EA9310E11A9317EFD9
:10930C0091221FEB9122E3E1F0E1B1E0BBBFB791F9
:10931C00BB2311F00E94225C10E11F9318810F9166
:10932C00011B102FFF91EF91108323960E94C62CE6
:10933C00DF91CF910C94A049FFCF11E01BBFF894A3
:10934C0018E005EC1EBF0DBF15B7106415BF112733
:10935C00E9E0F0E0A6E0B0E03196319711F01D9312
:10936C00FCCF1127E0E0F0E1A0E0B1E031963197BD
:10937C0011F01D93FCCFC8E8D9E0F8941FE79122B7
:10938C0009ED18E0280118E01093D90815E01093A6
:10939C00DA081093DB0806EC18E01093E40800934D
:1093AC00E30809EE18E01093E8080093E70810E0D2
:1093BC001093DE0810E11093E90813E01093EA080B
:1093CC001093EB0802E016E01093F2080093F108FA
:1093DC0002EB15E003501040F8011093F0080093D5
:1093EC00EF0803E016E01093F4080093F30809EF7C
:1093FC0018E01093F8080093F70811E01093EE08AA
:10940C0010E8119311930BE91DE11193008310E106
:10941C001093F90813E01093FA081093FB0802E17B
:10942C0018E010930209009301090EEA17E00350AB
:10943C001040F801109300090093FF0803E118E0B5
:10944C00109304090093030909ED18E0109308091F
:10945C000093070912E01093FE0810E81193119382
:10946C000EEB1EE3119300830E94356416E012BFCD
:10947C0015E013BF11E017BF112717B913EC16B97C
:10948C0018E11AB913E319B910E01093900010E029
:10949C00109367011093680110936901579A10E0BB
:1094AC0010930001109301011093020116E0109328
:1094BC0095001CB118E110939A0013E310939900D6
:1094CC0010E01093980010E01093350210933602C0
:1094DC001093370210919A00106810939A0010E0C4
:1094EC001093CE011093CF011093D00116E010937E
:1094FC009D0010919C00EEEAF2E010E000E8008381
:10950C00118313E0128317E0138310E0148310E02F
:10951C000FE10583168310E00FE10783108710E835
:10952C00118710E0128710E000E00387148710E029
:10953C0000E005871687EDEBF2E012E00DEE0087F8
:10954C00118712E00EEA0287138712E00DEC0687F2
:10955C0017871EEF1093EE0315EE1093AB0312E07A
:10956C000DEE0093B0031093B10300E81CE7EDEE91
:10957C00F2E011930A95E9F71127109371031093F8
:10958C00A60311E01093ED031FEF10936D031093DE
:10959C006E0310936F031093700310937203109368
:1095AC00740312E00DEE0093750310937603A0E0A4
:1095BC000E947E4F0E940556112715BB1FE714BB56
:1095CC0013E015BB00E111270E94295B15B3106154
:1095DC0015BB00000000000015B31F7E15BB05E095
:1095EC0011270E94295B15B3106115BB0000000008
:1095FC00000015B31F7E15BB01E011270E94295BEB
:10960C0015B3106115BB00000000000015B31F7EE0
:10961C0015BB12E015BB01E011270E94295B15B3A5
:10962C00106115BB00000000000015B31F7E15BBB8
:10963C0001E011270E94295B15B3106115BB0000D6
:10964C000000000015B31F7E15BB18E015BB01E030
:10965C0011270E94295B15B3106115BB0000000097
:10966C00000015B31F7E15BB1CE00E948A4C11E054
:10967C000E948A4C16E00E948A4C899800008898B7
:10968C009198000090989924AA240E942B080E947B
:10969C00BE2A0E94252C0E94922C0C944749EF93D1
:1096AC00FF930F931F931FB71F9316E002B7100F72
:1096BC0012BF1FE7912204B115B11F93E7B1E770F8
:1096CC00EF93F091AC02F17041F4E395E83008F0BF
:1096DC00EE27F7B1F87FEF2BE7B91F91110FECE9EB
:1096EC00F2E0E10F08F4F3951F910083118310E869
:1096FC00912A369A10918809112309F037C02F93BB
:10970C0022E0E9EEF8E003811481112311F4002327
:10971C0051F00150104014830383112321F40023D2
:10972C0011F410E110831081103229F411811123EE
:10973C0011F01A9511832A9511F07096E4CF2F91A0
:10974C00F20110811123E9F0110F58F0110FC8F03C
:10975C00110FB8F01181112381F01A95118369F062
:10976C0005C01181112311F01A9511831F911FBF90
:10977C001F910F91FF91EF91189510E110831281B9
:10978C0011830C94895A1895EF93FF930F931F93A1
:10979C001FB71F9310910201112311F4559816C095
:1097AC00009101011127E3E0F1E0E00FF11F1081BE
:1097BC001CB9109102011A951093020109F45598E5
:1097CC000395043609F40027009301011F911FBF74
:1097DC001F910F91FF91EF911895EF93FF930F93BA
:1097EC001F931FB71F931091D001112331F41091C7
:1097FC009A001F7D10939A001BC00091CF01112776
:10980C00E1EDF1E0E00FF11F108110939C0010913D
:10981C00D0011A951093D00129F410919A001F7D54
:10982C0010939A000395043609F400270093CF0196
:10983C001F911FBF1F910F91FF91EF911895EF93FF
:10984C00FF930F931F931FB71F9310916901143649
:10985C0011F41CB118C01CB11F93112700916701A2
:10986C00EAE6F1E0E00FF11F1F91108310916901FE
:10987C001395109369010395043609F4002700939E
:10988C0067015F99E2CF1F911FBF1F910F91FF914D
:10989C00EF911895EF93FF930F931F931FB71F939F
:1098AC0010913702143619F410919C001BC01091C2
:1098BC009C001F93112700913502E8E3F2E0E00FC2
:1098CC00F11F1F91108310913702139510933702DB
:1098DC000395043609F400270093350210919B0080
:1098EC0017FDDECF1F911FBF1F910F91FF91EF91BD
:1098FC0018951F9354D014B31F6714BB15B31F7E58
:10990C001079106215BB09C01F9349D014B31F679F
:10991C0014BB15B31F7E107915BB1F911F931295A5
:10992C001F7005B3012B05BB1F9100000000000048
:10993C00000000000000006105BB000000000000FA
:10994C0000000000000005B30F7E05BB0000000006
:10995C0000000000000000001F7005B3007F012B09
:10996C0005BB0000000000000000000000000061CA
:10997C0005BB00000000000000000000000015B353
:10998C001F7E15BB08950BD014B3107F14BB15B3F9
:10999C001F7E107F106615BBE89494F817C0E0E8A2
:1099AC00F2E0689494F802C0E89494F814B3107F31
:1099BC00106314BB15B31F7E1F7915BB000000008C
:1099CC000000000000000000106415BB0000000047
:1099DC00000000000000000015B3106115BB000072
:1099EC000000000000000000000003B30295007F9F
:1099FC0015B31F7E15BB0000000000000000000026
:109A0C00000015B3106115BB000000000000000041
:109A1C000000000013B31F70102B05B30F7E007FE6
:109A2C0005BB94FA0EF00895319719F0111F70F2DE
:109A3C0008951FEF0895FF91EF911F910F91EF93F0
:109A4C00FF93112311F41CE001C01DE0002309F069
:109A5C0012605ADF089518810981103011F410E852
:109A6C000DC0113011F410EC09C0123011F410E9D2
:109A7C0005C0133011F410ED01C010E8100F44DFD5
:109A8C00089511E041DF0895103011F410E80DC075
:109A9C00113011F410EC09C0123011F410E905C0AA
:109AAC00133011F410ED01C008951F932DDF10E158
:109ABC001F9310E21EDF1F911A95D1F71F9124DF1F
:109ACC00089512E021DF08959098000091988898ED
:109ADC000000899811E00E94395B899A11E00E947C
:109AEC00395B889A0895889A0000899A11E00E943F
:109AFC00395B889811E00E94395B899811E00E94CB
:109B0C00395B089558E0889A441F10F0899A01C077
:109B1C00899811E00E94395B8898002411E00E941A
:109B2C00395B0A9409F41DC010B310FBBEF75A95AB
:109B3C0051F7889A0000899811E00E94395B889847
:109B4C0011E00E94395B10B311FB1EF0889A1FEFD5
:109B5C00089588980000899811E00E94395B10E004
:109B6C00089588980000899811E00E94395B889AC2
:109B7C000000899A0000889811E00E94395B89984E
:109B8C0011E00E94395B10E0089538E089980000DC
:109B9C00889A11E00E94395B8898222711E00E9474
:109BAC00395B2A9509F4DDCF00B300FBBEF788942E
:109BBC0000B301FB0EF40894441F3A9549F7142F97
:109BCC0010833196889A0000899A689490F81197BE
:109BDC0031F40A2F002319F4E89490F8899811E0D5
:109BEC000E94395B889811E00E94395B889A11E0D9
:109BFC000E94395B90FA4EF21FEF0895412F0E949C
:109C0C006A4D8894441F0E94884DB12F0E94794D53
:109C1C001B2F08950E946A4D0894441F0E94884D82
:109C2C00112321F40E94794D10E008950E94CB4D30
:109C3C000E94794D1FEF08950E946A4D8894441F2D
:109C4C000E94884D112321F40E94794D10E0089553
:109C5C00432F0E94884D112321F40E94794D10E06E
:109C6C00089590FA4EF4422F0E94884D112321F44E
:109C7C000E94794D10E00895AA2311F4BB2319F02A
:109C8C0041911197F1CF0E94794D1FEF08951091DA
:109C9C00AD02112309F04CC0109169011123E1F3BD
:109CAC00F894009168011127EAE6F1E0E00FF11F4A
:109CBC001081009169010A95009369010091680176
:109CCC000395043609F400270093680197FC7894F7
:109CDC0008951091AD02112309F047C0112700918E
:109CEC006901002309F0109508950091AD0200233D
:109CFC0009F042C0009102010436E1F3F89400919E
:109D0C000001E3E0F1E0E00F0027F01F1083009169
:109D1C0002010395009302010091000103950436A2
:109D2C0009F4002700930001559A97FC7894089544
:109D3C00109137021123E1F3F894009136021127A8
:109D4C00E8E3F2E0E00FF11F1081009137020A9571
:109D5C0000933702009136020395043609F400276C
:109D6C000093360297FC78940895112700913702DE
:109D7C00002309F0109508950091D0010436E1F309
:109D8C00F8940091CE01E1EDF1E0E00F0027F01F17
:109D9C0010830091D00103950093D0010091CE0166
:109DAC000395043609F400270093CE0100919A0024
:109DBC00006200939A0097FC78940895F8940091AF
:109DCC009D000777103009F0086000939D0097FC08
:109DDC0078940895F89400919D000977103049F01B
:109DEC00113011F4026005C0123011F4046001C08E
:109DFC00066000939D0097FC78940895F894009168
:109E0C009D000F74103029F0113011F4006201C064
:109E1C00006300939D0097FC7894089522273327C4
:109E2C002093720330937303A2E0B0917103E22F7D
:109E3C00F32F5EC0FF27EE27213008F00895209302
:109E4C007103A1E0B22F54D0E0917103EE0FEE0F2D
:109E5C00EE0FEE0FE354FD4F089520937403A3E02F
:109E6C00B0917103E22FFF2743C020937503309309
:109E7C0076030895E22FF32F08950091C003069501
:109E8C0033271091720320917303110F221F331F7C
:109E9C000695D8F7369527951795E091740300270A
:109EAC00E6950795FF271E0F2F1F3F1F0895E5DF2F
:109EBC0000937703109378032093790330937A03FC
:109ECC00E0917503F0917603A4E0B091710310C09A
:109EDC00D4DF0093770310937803209379033093A6
:109EEC007A03E0917503F0917603A5E0B0917103CC
:109EFC00CF93DF93AA93BA93FA93EA933A932A9364
:109F0C001A930A930E94542BDF91CF9108950E94CB
:109F1C00F858002311F411270895E091AC03F09147
:109F2C00AD03212F3CD1E170B1F7EDEEF2E020E86A
:109F3C0005EE01932A95E9F71F93212F7BDF22274A
:109F4C0033276EDF222789DF2DEE32E08EDF1F9163
:109F5C00EEEAF2E0212F222319F03F962A95E9F739
:109F6C00A781B0851196B695A795B695A795103093
:109F7C0019F420E030E000C0A20FB31F0027CF93EC
:109F8C00DF930A930A930A93BA93AA93A1DFE88109
:109F9C00F9813197A9F0F983E8832A8123951091EF
:109FAC00C003211750F022272F932B813C812F5F68
:109FBC003F4F3C832B8334DF2F912A834EDFE6CF38
:109FCC001ED6DF91CF911FEF089528DF1127E09166
:109FDC00B403F091B50311931083E091B603F091A3
:109FEC00B703119310830895E091E903F091EA030C
:109FFC0022E0D5D0E093E403F093E503E093EB0388
:10A00C00F093EC03E4EEF3E021913081E091B603A0
:10A01C00F091B703A191B081E091B403F091B50335
:10A02C001191F081E12F2A173B0740F44091C003B6
:10A03C005091C103A41BB50B3197F5CFEF93FF9350
:10A04C00E091C003F091C103EA0FFB1F40F02E1703
:10A05C003F0728F0DF01FF91EF913196EFCFFF9191
:10A06C00EF912F933F93AF93BF93EF93FF93209177
:10A07C00CD033091CE032E0F3F1FD2DEBF91AF9197
:10A08C00E091B403F091B503A193B083BF91AF916C
:10A09C00E091B603F091B703A193B0833F912F9158
:10A0AC002A1B3B0BA091CF03B091D003E3DE9F01A1
:10A0BC00D4CEE2ECF3E020811091E2038894179562
:10A0CC002A95E1F7312F18E00081101B212F1091F8
:10A0DC00E1032A9519F08894111FFBCF130F0895F3
:10A0EC00E091A703F091A8037096E20FF31F109173
:10A0FC00DC03112319F0E081FF270895E20FF31F11
:10A10C00A191B081DF010895D4DF212F3327E8DF3F
:10A11C00E093E403F093E50308951091C203E091FA
:10A12C00E403F091E503EE0FFF1F1A95E1F7E093BE
:10A13C00E603F093E7032091C3031091E20312238B
:10A14C00E12BE093E403F093E5030895A091A703BA
:10A15C00B091A8031F96FD0171960895F7DF108149
:10A16C001093E2031C911093E003E091A703F0918C
:10A17C00A8033C961091C403008110231093E103B3
:10A18C000895E4DF1091D403123009F411270091E3
:10A19C00E203100F10830091E0030C9308952395B4
:10A1AC002A9509F40895F695E795FACF0091A60340
:10A1BC00FF27E1E003950A9511F0EE0FFCCFE22B9F
:10A1CC00F32B0895E091AC03F091AD032091A6031D
:10A1DC00E6DF1E2F117009F012E00895ECEAF3E0AF
:10A1EC0021913081E3DFE093AC03F093AD03E09178
:10A1FC00C703F091C8033196A091B203B091B30399
:10A20C00ED93FC93089508D039961081111F10F02E
:10A21C001127089513E00895E091B803F091B90364
:10A22C001091E8030027E10FF01F0895E091A703B8
:10A23C00F091A8033E9610810895F8DF0027008363
:10A24C000895F4DF106810830895A091E903B0918C
:10A25C00EA03E091B203F091B3031A2F0191101BA2
:10A26C001B2F0081100B0895F0DF08F40895119650
:10A27C00B0833197A08308951A2F1E1BE12F1B2F3B
:10A28C001F0BF12F08952FEFA091EB03B091EC036E
:10A29C00E091CB03F091CC03EFDF08F0089500E8D8
:10A2AC00E091B803F091B90311274191140F0A956D
:10A2BC00E1F7A091BC03B091BD03E091EB03F091E9
:10A2CC00EC03EA0FFB1F239549F00081101709F4EA
:10A2DC000895BBDF08F0089581DF08951083089579
:10A2EC00D2DF08D021E0F4DD02C004D0E0DDE0EBE9
:10A2FC00F3E002C0E8EBF3E021913081B6CDE9EE5A
:10A30C00F3E011910081101709F008951395089549
:10A31C00A091C703B091C803E091E903F091EA035F
:10A32C003196E093E903F093EA03A6DF38F4EFEFFC
:10A33C00FFEFE093E903E093EA0308951091E9033A
:10A34C00137035E0110F3A95E9F71093E8031123D8
:10A35C0009F008952F933F9347DEC7DF3F912F916C
:10A36C0093CF122F17701395A12FB12F26952695E9
:10A37C0026952F71132F110F110F110F110F110F94
:10A38C00212B3695369536953F71E091BE03F091B1
:10A39C00BF03E20FF31F1081110F08F41160AA958F
:10A3AC00D9F70895AF93BF93DCDF1E7F3F912F91B8
:10A3BC00122B169508F41068BA95D9F710830895E6
:10A3CC002BDF70962F933F9321E1BF91AF912A958C
:10A3DC0009F40895AF93BF931091DC03112339F066
:10A3EC002F933F93EF93FF932081332707C02A9538
:10A3FC002F933F9321913081EF93FF93122F132BC7
:10A40C0051F0E091C503F091C6031E2F121B1F2FB4
:10A41C00130B08F0C7DFFF91EF9131963F912F910D
:10A42C00D4CF1FEF1093D3032093D703E091A7034E
:10A43C00F091A803E093D803F093D903EFEFFFEF6B
:10A44C00E093E903F093EA03C0DD222761DF57DFD5
:10A45C0009F445C0FD01A091D803B091D9031C911A
:10A46C00153E31F0AF93BF93F0DEBF91AF91B8F5CD
:10A47C00D3DE2091D7033327222319F11C911F33EC
:10A48C00D9F03D30C9F03C301C9129F00081101BF3
:10A49C001F77D9F611C02F933F9320812F933F93B1
:10A4AC003091C403309523231323121B1F713F914A
:10A4BC002F913F912F9149F61196319633952A950C
:10A4CC00DBCF1091E90313701093A903E3EDF3E0D4
:10A4DC001081111F08F00895112710830895EFEFD4
:10A4EC00FFEFE093E903E093EA031FEFB2C420E02F
:10A4FC00A0E2B0E0AF93BF9330E0A091A703B0917E
:10A50C00A803A20FB31F88DE3F912F910D910193E9
:10A51C002A95E1F769DDE4CE2CE083DFF0DE09F467
:10A52C00089520E0ACE0E6DF90DFF8CF2FE079DF94
:10A53C00E6DE11F411270895E091A703F091A8032A
:10A54C003C9610811F93EF93FF9366DEA091A703B7
:10A55C00B091A80320E23327EF93FF9301910D9361
:10A56C002A95E1F76EDEFF91EF9124853785FF91F7
:10A57C00EF911F91108300812017132F19F01127D1
:10A58C0008F010E8E091A703F091A80317871038A2
:10A59C0011F4112715871FEF089510810181102BDD
:10A5AC0009F008951D9110831C9111831197089542
:10A5BC0011271093A9031093E9031093EA0302DE09
:10A5CC0009F0089533DE107841F0E091A703F09183
:10A5DC00A8032585222309F408952FE022DF8FDEBE
:10A5EC0009F4089520E130E017DEE20FF31FDF01DC
:10A5FC00E091A703F091A803E20FF31F20E1109163
:10A60C00DC03112369F0108111231C9109F41083D0
:10A61C00112311F410811C930081101781F517C0C0
:10A62C00BCDFEF93FF93FD01BF91AF91B6DFEF93CA
:10A63C00FF93FD01BF91AF911C9100811017F9F4AC
:10A64C00119631961C9100811017C9F42A95119618
:10A65C0031962A95A1F67497549710810C91101786
:10A66C0050F01D93118111230AF411271C9312969B
:10A67C00339610811C931FEF1093D1034BCFE9EA53
:10A68C00F3E000810A95008308959CDDE091A70317
:10A69C00F091A803EF93FF93EBEAF3E0E093A703A9
:10A6AC00F093A80321E0BDDE2ADEFF91EF91E09349
:10A6BC00A703F093A80311F411270895DF013F9627
:10A6CC0021E1112711932A95E9F7EA2FFB2F3D96EB
:10A6DC001083CADD0CDFB5CD11271093D10368DFD1
:10A6EC000EDE09F40895E091A703F091A8033C96BF
:10A6FC00108113951F71108351F0312F1091C403E9
:10A70C001323E1EDF3E00081102339F012C03296EF
:10A71C001081139510831F7081F02FE082DEEFDD26
:10A72C0041F41091D203139541F0AFDFE8DD29F02D
:10A73C0001C002DF13DD11278CC38AD382CD11E057
:10A74C001093D4031FEF1093D20308DD1091E20392
:10A75C00E0EEF3E00081101750F01038A1F4BCDFEC
:10A76C0011271093E2031091A903112361F4CCDC9F
:10A77C00E091E403F091E5031E2F1F2B21F0CDDCBB
:10A78C0041DC95DBFECC64C311E01093D40310E0E4
:10A79C001093D20317DDE091A703F091A80334DDE9
:10A7AC00DDDC1091E203103808F052C3ADDCE0910F
:10A7BC00E403F091E5031E2F1F2B20E009F065C088
:10A7CC0078DC1093D60320E030E0112331F0212FF8
:10A7DC002150304085DC3F2F2E2FB32FA22F122F6C
:10A7EC00132B69F021503040AF93BF932F933F93BD
:10A7FC00B8DD1695E0F43F912F91BF91AF91E091A8
:10A80C00C503F091C6031A2F1E1B1B2F1F0BB8F488
:10A81C0011962F933F93AF93BF933B2F2A2FA1DD1C
:10A82C00179528F4BF91AF913F912F91D8CF111F5D
:10A83C001395BFDDFF91EF91BF91AF9105C0122F22
:10A84C00132B69F6E0E0F0E01E2F1F2B11F412E041
:10A85C0000C3E093E403F093E503DF01E091A70369
:10A86C00F091A80370961091DC0311231091D6037C
:10A87C0019F0D8DCA08308C0212F3327E20FF31F77
:10A88C00E20FF31FA193B08322E01091A9031123CF
:10A89C0009F008952F933F9340DC1091D40312508C
:10A8AC00A1F53F912F912F933F93122F125069F5E1
:10A8BC00EF93FF93E091B803F091B903B12F11938B
:10A8CC00B395EAF717DDE091E603F091E70322E098
:10A8DC00E093E403F093E5032F933F9393DB3F91D5
:10A8EC002F91F6DAE091E403F091E50320E010916A
:10A8FC00C303312F1E233196131751F7FF91EF919C
:10A90C00E093E403F093E503F2DC7CDB3F912F91C1
:10A91C002F933F93DDDA3F912F911091E203E0EEFC
:10A92C00F3E00081101720F0012F0395008322E043
:10A93C00225029F41F937ADC1F7710831F911F3745
:10A94C0081F41091D403113061F41BDCC5DEE9EA0B
:10A95C00F3E01081112319F41A951093E2030027E8
:10A96C0000830FCC11271093D4032F933F93E091C6
:10A97C00A703F091A803DF0111A11F771F9311A169
:10A98C00111F12A1111F1F77212F12A117951795B7
:10A99C00179517951F70312F1F9103A10023E6E027
:10A9AC00C1F5FD0110A3122F0485101B29F4132FE0
:10A9BC000685101B1F7711F12F933F93AF93BF9315
:10A9CC00F7DDBF91AF913F912F91E3E01091A90377
:10A9DC001395C1F0EA2FFB2F24873687A7DD1123AF
:10A9EC0069F43F912F912F933F93E4E0239551F01D
:10A9FC004CDEE5E0E091A903139521F03F912F91F6
:10AA0C00112727C2EF93FF9311DC00EC0083FF9119
:10AA1C00EF913F912F91122F1093A90312CCEF932A
:10AA2C00FF93FD01BF91AF91EA0FFB1F20813327EC
:10AA3C00EA2FFB2F1485179517951078210F1127E6
:10AA4C00311F148517951F70310F1685110F110FBB
:10AA5C00110F110F1F93130F312F11E008F010E09D
:10AA6C00EF911E2B11700895A0E2B0E0D8DFEA2F11
:10AA7C00FB2FB1962193319310830895E091AE038F
:10AA8C00F091AF032091A6038ADBEF93FF93FD01B6
:10AA9C002091A603CFD91F2F1E2B99F1A191B19113
:10AAAC00E093B203F093B3033296E093B403F093C4
:10AABC00B5033296E093B603F093B7033296A093A6
:10AACC00CF03B093D003A8EBB3E028E001910D9332
:10AADC002A95E1F7E091BA03F091BB03A0ECB3E047
:10AAEC002FE001910D932A95E1F71091C603ECED3F
:10AAFC00F3E00FEF0083112311F000E000831FEF50
:10AB0C001123FF91EF911E2F179508F408952091B2
:10AB1C00AE033091AF034ADBE093AE03F093AF0387
:10AB2C00E091C503F091C60323E039DB3196BF2FCA
:10AB3C00AE2FE091BE03F091BF0300270193119754
:10AB4C00E9F7A091C903B091CA03E091BE03F0915B
:10AB5C00BF03A193B08339DAE091B203F091B30350
:10AB6C0003E0019300E000830FEF0093E9030093EF
:10AB7C00EA032FEFCDDBC3DB09F408954DDB108125
:10AB8C00153EB9F321E01CDC6FDBF3CF1FEF109304
:10AB9C00DD03E091A703F091A80310811F711A95B2
:10ABAC001093D5031E3150F41091A6031093DE03BD
:10ABBC0010811093DF03107E108317D0E091A70350
:10ABCC00F091A80314A10081011710830895A0919E
:10ABDC00B003B091B103E091B803F091B90320E850
:10ABEC0001910D932A95E1F708951091D5030091E9
:10ABFC00A603011709F408951093A6033FCF2CD197
:10AC0C0010E01093AC031093AD031093AE031093AC
:10AC1C00AF031093A603EDEEF2E0E093B003F093D4
:10AC2C00B10365DB2BCF18D1E0CF16D106DBAEDF3D
:10AC3C007DCC12D1ABDFBCCC0FD120E01C911F33EB
:10AC4C0051F0E091A703F091A80314851F3309F08C
:10AC5C00F4DA9CDF2FE0E5DBBACFFED0E091D8032D
:10AC6C00F091D903E093A703F093A8038FDFEDDBFA
:10AC7C00AECFF2D08BDF2CE0D4DB1091D303109548
:10AC8C0009F01FEFE6C0E8D081DF9CDA2CE0C9DBCD
:10AC9C0036DB49F0B8DAC0DA05EE008320E090DB51
:10ACAC001FDBD3DBF5CF1091D303D3C0D5D06EDF30
:10ACBC0046CDD2D06BDF68CDCFD0BFDA67DFE5CC25
:10ACCC00CBD0E091AE03F091AF031BC0C5D0109177
:10ACDC00A603BFC0C1D0A093B003B093B10307CB00
:10ACEC00BBD0E091BE03F091BF030BC0B5D0E09197
:10ACFC00AC03F091AD0305C0AFD0E091BA03F09175
:10AD0C00BB03A093A903B093AA030895A5D01091F7
:10AD1C00D5031F3F19F41091A5039BC01F71A0937D
:10AD2C00A503089599D032DF2FEF1CDE11F0112707
:10AD3C00089508DD0091A903002349F1E091A703D0
:10AD4C00F091A803002700A3048701A302A303A387
:10AD5C002CD0E091A703F091A80301A1015001A30D
:10AD6C0002A1004002A303A1004003A338F4112761
:10AD7C0010A3148711A312A313A30895002704870B
:10AD8C0000A356A155A3DF01CDDF1FEF0895E0917D
:10AD9C00A703F091A8030091E203039500A300918F
:10ADAC00E00307871FEF089557D0F0DE2CE039DB66
:10ADBC00E091A703F091A803B196EF93FF9300E005
:10ADCC000193019300839BDAD1F026DA8585AFE0FD
:10ADDC00B0E025DEFF91EF91EF93FF938583A12FD8
:10ADEC00122F0191101B132F0191100B1A2F01918F
:10ADFC00100B18F0A2933293229327DBE4CFFF9130
:10AE0C00EF91089529D0A091A703B091A803A09524
:10AE1C00B095E091AE03F091AF03BF23AE23E09168
:10AE2C00AC03F091AD03A093AE03B093AF03AE238C
:10AE3C00BF23A093AC03B093AD0308950DD0A6DE51
:10AE4C0012E01093D40320E090DD09F4A0DC089507
:10AE5C0011E01093A9030895A093A703B093A8033E
:10AE6C00A093D50311271093A9031093AA03109351
:10AE7C00DF031093DD030895EBE7F3E0EF93FF930B
:10AE8C003091ED032091A503A091A303B091A403ED
:10AE9C00FD0111911123E9F001910023D1F00A3346
:10AEAC0029F041914423A9F04A3399F4DF0110337E
:10AEBC0068F01A3371F040F01F7D113438F01534FE
:10AECC0028F41770312F02C01053212F102F042F8C
:10AEDC00EECFFF91EF91EF93FF9324A3308338E0F3
:10AEEC001FD033E01E3211F02CD002C0119618D0B6
:10AEFC0033E000E0319600833A95E1F7A093A30389
:10AF0C00B093A403FF91EF913BE020E031961191B7
:10AF1C001F3309F423953A95D1F7122F1123089575
:10AF2C0016D079F031961A3219F40FE3008302C06F
:10AF3C00108311963A95A1F70AD009F40895119649
:10AF4C00FBCF319600E200833A95D9F708951C9116
:10AF5C00112399F0103289F01D3379F01E3269F00B
:10AF6C001A3359F01B3349F01B3539F01D3529F0D4
:10AF7C001C3219F01C3309F01E330895FE01709633
:10AF8C00DF010191002379F005C0FE01DF01019181
:10AF9C00002349F01081113618F01B3708F41052B9
:10AFAC0011930A95B9F7FD0101910F3028F411277F
:10AFBC00DF01A00FB11F1C93E093A303F093A40334
:10AFCC000895E3EFF3E0A8EAB0E018E001E0209187
:10AFDC00EE03322F302331F0EA0FFB1F000F1A95CE
:10AFEC00C1F70895202B2093EE03DF019F0118E297
:10AFFC0000E00D931A95E9F71FEF089523EF33E066
:10B00C0048EA50E018E061E02E173F0731F0240FBA
:10B01C00351F660F1A95C1F70895DF011FEF0895CC
:10B02C00EDDF112331F07091EE036095672360938F
:10B03C00EE030895A6E0B0E00E947E4FE0DD1EEF27
:10B04C001093EE0301E00093ED0308959EDF14DFEF
:10B05C00ABE7B3E00EDE109509F40895ABE7B3E06F
:10B06C0011271C9329DE112309F40895EBE7F3E073
:10B07C0010E015A316A3DF01DCDD089586DFFCDEEE
:10B08C00ABE7B3E000DE1091A903139509F01FEFB5
:10B09C00089597DF112309F40895EF93FF931ADEB7
:10B0AC0074DFFF91EF91EF93FF93E8DEBF91AF91C7
:10B0BC00AF93BF93BADDFF91EF91112389F0A8896B
:10B0CC00B989ED93FD93B0E0B5A3A785A23010F03C
:10B0DC00B0E001C0B585B6A31FEF1093D20308955D
:10B0EC009FDFE889F9891127108311830895A881BE
:10B0FC00B981ED91FD9182DF112309F40895EF934D
:10B10C00FF9307A1002361F0FF91EF91DF01EF9313
:10B11C00FF93078510A1011711F405A10587C9DD5F
:10B12C00BF91AF91AF93BF9384DDFF91EF9178DF27
:10B13C00A6E0B09171030E947E4FE881F98111273E
:10B14C00108311831095089520DF96DEABE7B3E0F2
:10B15C0073DD1091A903143028F4E889F989FA9366
:10B16C00EA9314C01127E889F98910830895ABE795
:10B17C00B3E010E01C9371DD1091A903143008F4B6
:10B18C0005C01127E881F98110830895ADEEB2E076
:10B19C0000271295110FA10FB01FFD011285107819
:10B1AC0031F71196E881F981319628E01D911F77CE
:10B1BC00103211F0039511932A95C1F71C9110329E
:10B1CC0061F01EE21193039523E01D911F7710325D
:10B1DC0021F0119303952A95C1F7E881F981008339
:10B1EC001FEF0895113618F01B3738F41052115414
:10B1FC0020F0113010F40FEF089500270895F2DFBE
:10B20C00002329F400E010E020E030E008951F93C3
:10B21C00A12F09DDE091BE03F091BF03A0E0B0E0E7
:10B22C0050E248E01191111F08F411964A95D9F794
:10B23C005A95B9F71F91103019F410E000E200C0D4
:10B24C000A1B1B0B4091C20342504A9519F0000F88
:10B25C00111FFBCF0895F801D1DE112311F41FEF5C
:10B26C0008951785112339F000A1011730F016A1AC
:10B27C0005A1101710F01FEF08951127089500E095
:10B28C0010E020E030E00895EE81FF81B7DE11235D
:10B29C00B1F307A1002339F010E815A310E007A3C0
:10B2AC00AE81BF8106DD3B812A811981088160E076
:10B2BC0070E04C815D810E94C662402F012F122FDD
:10B2CC00232F440F001F111F221FC8F24695EE8139
:10B2DC00FF8101A312A323A30027048700A350E836
:10B2EC00541B55A3DF011EDDEE81FF8130E010A160
:10B2FC000785101718F0103809F0358536A310E0C3
:10B30C001093D2034C815D815A934A930DD04FEF29
:10B31C004093D2030895EA81FB8170DE112309F476
:10B32C000895A2DBEA81FB81442751A162A173A19C
:10B33C0076956795579547951091D203112349F44B
:10B34C0015A100E8011B1127400F511F611F711F30
:10B35C000CC005A11127401B510B610B710B28F47C
:10B36C0000E010E020E030E00895A881B981E0E031
:10B37C00F0E0E89495F80E941263882331F0992745
:10B38C0081E0080F191F291F391F0895EC81FD81D9
:10B39C0035DE112309F4089507A1002339F010E8D4
:10B3AC0015A310E007A3AC81BD8183DC1FEF1093C4
:10B3BC00D203EC81FD8156A1288139812F933F93D3
:10B3CC00AC81BD8195961D9112961123A9F0002791
:10B3DC00212F21952F77A20FB01FEA81FB812881A5
:10B3EC003981511738F40D9101932150304081F17E
:10B3FC001A95B9F739832883AC81BD8157DC288134
:10B40C0039810091A9030023F9F4EC81FD8150E00E
:10B41C0040A10785401720F0403811F0558556A300
:10B42C0010E8AC81BD819896EA81FB81511760F4DC
:10B43C000D9101932150304059F01A95B9F7FB83C7
:10B44C00EA8339832883D8CFEC81FD8116A113952B
:10B45C001A95EC81FD8115A300E007A35F914F9134
:10B46C00421B530B598348830895EC81FD81C6DD43
:10B47C00112309F4089510E01093D203AC81BD811F
:10B48C0095961D911296112391F00027212F21954D
:10B49C002F77A20FB01FEA81FB812881398101919E
:10B4AC000D9321503040E1F01A95C9F711C0AC81D1
:10B4BC00BD810FEF97960D93EA81FB81288139812D
:10B4CC0010E801910D932150304051F01A95C9F7B5
:10B4DC00AC81BD81FB83EA8339832883EADBE7CF28
:10B4EC00398328831A95EC81FD8115A3112319F05A
:10B4FC001FEF17A3089510E815A310E017A3AC8154
:10B50C00BD81D7DB08950E94DE5AF2010DB71EB73C
:10B51C000683178306851785F80110811123D1F353
:10B52C00110F78F0110FB0F3110F18F0110F38F054
:10B53C00F1CF04851585D8011C91112359F318E01E
:10B54C0010832F01178106811EBF0DBF0E94035B64
:10B55C006F906FBE1895F894F20110E1108306C03D
:10B56C00F894F20110E40081101711F0128111838C
:10B57C000F931F930F931F931FB71F930C94895A0C
:10B58C000895DF01F894F20110E21083B587A487C7
:10B59C00348323830E94BE5A1FEF08957F906F90CF
:10B5AC00EF93FF930F931F931FB71F93F20102C0EA
:10B5BC007F906F90D187C0878F9013850285F8019B
:10B5CC001F910F911193019331932193B193A193F7
:10B5DC001F910F9111930193519341937193619327
:10B5EC009192019291938193119231922192E894CC
:10B5FC0097F88F92F3010994F201D185C0851385D8
:10B60C000285F80111911F93019131912191B19112
:10B61C00A19111911F9311911F935191419171918E
